:040000006F00204429
:100004000000000000000000480200004A02000056
:100014000000000040040000000000000000000098
:100024004004000040040000000000000000000044
:10003400DE1C00000000000040040000000000007E
:10004400400400004004000040040000400400009C
:10005400400400004004000040040000400400008C
:100064006A1700004004000040040000400400003F
:10007400400400004004000040040000400400006C
:10008400400400004004000040040000400400005C
:10009400400400004004000040040000400400004C
:1000A40040040000EC1C0000400400004004000078
:1000B400C21C0000121C00004004000040040000A8
:1000C400400400004004000040040000400400001C
:1000D400400400004004000040040000021B000033
:1000E4000618000040040000400400004004000022
:1000F40040040000481B00004004000040040000CD
:1001040040040000400400004004000040040000DB
:100114004004000000000000000000000000000097
:1001240000000000000000000000000000000000CB
:0C013400000000000000000000000000BF
:10014000397101436EC619A0397141536AC866CA34
:1001500062CC5ECE19A0397101535AD056D252D416
:100160004ED64AD826DA22DC06DE3301614082828E
:1001700041114AC026C222C406C68282B24D410144
:10018000024D924C224CB24B4101024B924A224A00
:10019000B2494101024992442244B2404101828065
:1001A0003D432A876373C3029377F700BDEFADE544
:1001B000937606FF3D8ABA960CC34CC30CC74CC756
:1001C0004107E36BD7FE11E28280B306C3408A0683
:1001D0009702000096966780A6002307B700A30643
:1001E000B7002306B700A305B7002305B700A30493
:1001F000B7002304B700A303B7002303B700A3028B
:10020000B7002302B700A301B7002301B700A30082
:10021000B7002300B700828093F5F50F9396850011
:10022000D58D93960501D58D61B7939627009702DA
:10023000000096968682E78086FA9680C1171D8F09
:100240003E96E374C3F8A5B701A001A0EFF25FF2F8
:100250000545EF0010299922EF10F03E7165130556
:100260000520EF10B043B707002083A58716378518
:10027000000013054545EF6050291925AA853785EB
:10028000000013054546EF605028EF402007EF308F
:10029000707D014501B7EFF2BFED371402401C40FD
:1002A0003707FF08411193E717001CC05C40F98F26
:1002B0005CC01C403707F7FE6D17F98F1CC01C404F
:1002C0003707FCFF7D17F98F1CC05C40370701FF23
:1002D0007D17F98F5CC0B7079F001CC4EF00700743
:1002E00002C402C6B7270240054798C31C404167B5
:1002F000B7160240D98F1CC03706020005679C4222
:10030000F18F3EC6A24785073EC4B24781E7A247A8
:10031000E397E7FEB71702409C431397E700635744
:10032000070685473EC6324785476313F706B7176A
:100330000240D843B706C1FFFD16D8C3D843D8C37F
:10034000D84313670740D8C3D843758FD8C3D84361
:10035000B7061100558FD8C39843B7060001558FD3
:1003600098C3984393166700E3DD06FED843B7169B
:100370000240719BD8C3D84313672700D8C32147D5
:10038000DC42B18BE39EE7FE410129B502C661BFA5
:10039000372702401C43F19B1CC3FDB7B716024030
:1003A000DC42370700201146B18B13078716638F95
:1003B000C70221466381C70495EB9C42918B9DC780
:1003C000B7470F00938707241CC3B7170240DC43CD
:1003D000918393F6F700B707002093870700B6973D
:1003E00094231C43B3D7D7001CC38280B7177A006D
:1003F00093870720D1BFDC42D4424166C983BD8BBD
:10040000F18E890745466393C700C94781EEB74619
:10041000024083A60680C18A89CEB7167A009386E9
:10042000062021A8B7160240D4421396E600E356F0
:1004300006FEB7163D0093860690B387D70269B7CC
:1004400001A09701002093816152175100201301F0
:1004500061BB179500001305E5A99705002093855A
:1004600065BA1386018263FAC5008322050023A0C2
:10047000550011059105E3EAC5FE13850182971524
:1004800000209385A50A6377B50023200500110598
:10049000E36DB5FEFD42739002BC8D4273904280C5
:1004A0009302800873900230970200009382C2B5D5
:1004B00093E2320073905230EFF0FFDD97020000BC
:1004C000938202D97390123473002030B727014011
:1004D00093870740631FF500EFF29FC98545130519
:1004E0000020EF001018814513050020EF00701761
:1004F00055B182805C413707F1E01307F7EF944D67
:100500007D8F9C41D58FD44DD58FD441A206D58FF8
:10051000D98F5CC11C4537F7F1FF1307D77FD4454E
:100520007D8F9C49D58F94458606D58FD98F1CC564
:100530005C55370710FF7D177D8FDC29FD1793F77A
:10054000F70FD207D98F5CD582801C4589C593E708
:1005500017001CC58280F99BEDBF1C4593E78700FF
:100560001CC5828008450D81058982801C4593E762
:1005700047001CC5828008450981058982801C4589
:1005800091C537075000D98F1CC582803707B0FF4F
:100590007D17F98FD5BFA54763F7B7048D4713873C
:1005A00065FF3307F7020328C5009D47B397E700AF
:1005B00093C7F7FFB3F70701B396E600DD8E54C586
:1005C000994763E3C70495477D163306F6025859E9
:1005D000FD47B397C70093C7F7FFF98F3396C50060
:1005E0005D8E50D982800D473387E50203280501CF
:1005F0009D47B397E70093C7F7FFB3F70701B3969B
:10060000E600DD8E14C96DBFB14763E2C7029547AE
:1006100065163306F6021859FD47B397C70093C70E
:10062000F7FFF98F3396C5005D8E10D9828095470C
:100630004D163306F6025855FD47B397C70093C7CA
:10064000F7FFF98FB395C500DD8D4CD582806845E5
:1006500042054181828008416D8D3335A000828042
:100660005C4191C537070004D98F5CC18280370790
:1006700000FC7D17F98FD5BF3C4989C593E7070872
:100680003CC9828093F7F7F7E5BF3C4989C593E7FA
:1006900007043CC9828093F7F7FBE5BF3C4993F719
:1006A000F7FD3CC93C49DD8D2CC98280EFF25FAC7F
:1006B000B7066745B7270240938636123797EFCDC6
:1006C000D4C31307B79AD8C3D4D3011198C7D45B46
:1006D0001387470313962600E34B06FED4573725AE
:1006E00001401305054093E60620D4D7DC5BB7062E
:1006F0000020D58F1CC31C431C4537070E00D98F23
:100700001CC51C4593E717001CC53C4993E707042B
:100710003CC91C4593E787001CC52A84228599356E
:1007200075FD37250140832785401305054093E774
:1007300047001CC52A8422853D3D75FD37250140B3
:100740000546C945814613050540B13525462304B4
:10075000010037270140B70550001C84637FF60471
:1007600023040100A54621461C8463FFF6062315D9
:1007700001002304010095461C8463F1F60E3885C0
:100780003C8599460D46B3F7D702056513050580EC
:100790003357D702B3D7C702BA97C207C1837C8544
:1007A000B727014003A78740799B23A4E7403C85F6
:1007B00005611D8D42054185F1BA83278740CD8FA4
:1007C0002324F74083270740898BEDDF1C84832691
:1007D000C74408108607AA972396D7FE1C8485076E
:1007E00093F7F70F5C8495BFA30401009C846378A2
:1007F000F6001C84850793F7F70F5C84B5B79884DF
:100800009C840C100607850786072E97AE97035722
:10081000C7FE83D7C7FE63FDE7029C848607AE97B9
:1008200083D7C7FE7C859C84988485078607AE970E
:1008300083D5C7FE931717001810BA972396B7FEF3
:100840009C8438850C1085078607AE972396E7FEB3
:100850009C84850793F7F70FDC8449BF1C84101034
:10086000388589078607B29783D7C7FEBA97C2072C
:10087000C1837C851C84850793F7F70F5C84EDBDED
:1008800003A5418282805841032805004C45370664
:100890000140930706403E979346F8FFB1C5832574
:1008A0000640F58D2320B640D043F18ED4C31443C7
:1008B000B3E6060114C3184190479346F7FF758EBF
:1008C00090C7D047F18ED4C7144541466399C600FE
:1008D0009447D98E94C7D447558FD8C78280B6978E
:1008E0009443558F98C382801C43F58F1CC382802C
:1008F000B70701401387074083A70740584B698F0C
:1009000009C77D8D3335A000828001458280B707FD
:10091000014023AAA74082809C4513F7070113F8E2
:10092000F70001C7D8413368E8008E2113F7F50FAF
:1009300039C318418146854E3D4F930F8002930283
:100940008004214E3396DE00B3F8C5006311160310
:100950009398260033131F011343F3FF3377E3000B
:10096000B318180133E7E800639FF70550C98506FF
:10097000E39AC6FD18C11307F00F6375B70454411D
:100980002146854E3D4F930F800293028004414ED5
:10099000B398CE0033F715016392E80213172600CF
:1009A00001173313EF001343F3FFB376D30033176C
:1009B000E800D98E639DF701232A15010506E31986
:1009C000C6FD54C18280E39457FA10C94DB7E3972E
:1009D00057FE23281501DDB708456D8D3335A0007E
:1009E000828048456D8D3335A00082800CC982809D
:1009F00019C20CC982804CC98280370700C0B37706
:100A0000E5006395E708370701405C439356B5015D
:100A1000584F9D8A9DE6F99BB70600FFFD16758F1E
:100A200089C993160501C182D58FB706FF01758D5F
:100A3000498FB7060007D58FB7060140DCC2D8CE74
:100A4000828005466396C600F59BB70680FFF9B71E
:100A500009466396C600ED9BB706E8FFC1B70D4691
:100A60006396C600DD9BB706FCFF4DBF114663973A
:100A7000C60093F7F7F3B706C0FF4DB71546E391ED
:100A8000C6FA93F7F7CFB706E0FF49BF3707004034
:100A90006391E702B7070140D84F4205B367A7004B
:100AA00089E51345F5FFB377E500370701405CCFD3
:100AB0008280A9E337080140B707300003264800C9
:100AC00013170501B376F50041836396F602B70666
:100AD00000F9FD16B377D60003264800F18E2322D5
:100AE000D80091C5558112053315A700C98F370766
:100AF00001405CC382809317B50063D0070293570F
:100B0000050193F6F7008D47B397D70093C7F7FF1A
:100B1000F18FB7060007D58FE9B7935755019207B4
:100B2000B317F700E5B713F7C50F93F73500B7050F
:100B30000140BA9594458A073D473317F70013479C
:100B4000F7FF758F98C598453315F500598D88C501
:100B50008280EFF2EFE137F4FF1F0327447237067C
:100B6000003E4111931797019346F7FFF18F060757
:100B700037063E00718FD98F370600011397960014
:100B8000718FD98FBD824167F98ED58F02C202C4A1
:100B900002C623A4F1820357847285452390E18223
:100BA000032704721305D00323A6E18203274470B0
:100BB00023A2E1828D2C8327447037073A10130754
:100BC000077093F7F7F06380E7106361F702370768
:100BD0003210130707706380E706370737101307D3
:100BE00007706387E70841016FF0CFDA37073B10E2
:100BF00013070770638BE70A37073D101307077069
:100C0000E393E7FE85452165CD3BB7140140E177CD
:100C1000130480044C00138504807C8222C6ED39C5
:100C200085679387C7334C00138504C07C8222C636
:100C3000E531F9770DA085452165C133B714014031
:100C4000930700E0130480044C00138504C07C82E9
:100C500022C6D93189674C00371501407C8222C6F3
:100C600065398D477C8222C64C001385044025A837
:100C7000B7140140E17793870770130480044C0098
:100C8000138504807C8222C641399307D0E34C004F
:100C9000138504C07C8222C64131F9777C8222C64A
:100CA0004C00371501408D393DBFB7140140E17745
:100CB000130480044C00138504807C8222C6A93969
:100CC000930740208DB7B7140140E17713048004E7
:100CD0004C00138504807C8222C63D398967F51754
:100CE00099B723A8A182828003A701838547142195
:100CF0006310F7021C31639CE7023C21960793E7DF
:100D000007F837E700E093F7F70F36972300F7402F
:100D1000054793D756003317D700544189CE9387A0
:100D200007048A07B7E600E0B69798C38280EDF320
:100D30003C219607F9B793870706E5B7B716024037
:100D4000DC423747FF7F7D17F98F5D8DC8C28280F7
:100D5000371702405C439146B18B638CD706A1469E
:100D6000638ED706BDE71C43918BA5C7B7470F001D
:100D7000938707241CC1371602405C4237070020C6
:100D8000130707019183BD8BBA9794231C41B3D7F6
:100D9000D7005CC15442A1829D8ABA969422B3D6F0
:100DA000D70014C55442AD829D8A36971423B3D61A
:100DB000D70054C55842634C07005C42B98313F70F
:100DC000370093874180BA979C23B3D7F6021CC99A
:100DD0008280B7177A009387072069BF5C43584326
:100DE000C166C983BD8B758F8907C5466393D700DC
:100DF000C94701EF3747024003270780418B09CFDE
:100E000037177A001307072021A8371702405843E5
:100E10009316E700E3D606FE37173D001307079049
:100E2000B387E70281BF99C5371702401C4F5D8D1C
:100E300008CF8280B7170240984F1345F5FF798D90
:100E400088CF828099C5371702405C4F5D8D48CFAF
:100E50008280B7170240D84F1345F5FF798DC8CF70
:100E6000828099C5371702405C475D8D48C78280F4
:100E7000B7170240D8471345F5FF798DC8C7828060
:100E80001A218D6793870704B6217D8F9E21D58F08
:100E9000D621D58FF621D58F9625D58FB625D58F1E
:100EA000D625D58FF625D58FD98F1EA19E291EA9AF
:100EB00082801E2189C593E707041EA18280C20794
:100EC000C18393F7F7FBC207C183C5BF4EA58280DC
:100ED0004A2582800A256D8D3335A00082801E212F
:100EE00037370140130707C0C207C1836300E5021B
:100EF00037070040630CE500130707406308E5006F
:100F000037170040130707806316E500FA2193F7AF
:100F1000F7F8D98F9A2593F7F7CFC207C183D98FF6
:100F2000371700401EA1130707809C416310E5029C
:100F30005CD5DE211EB5B7370140938707C0631427
:100F4000F500BC251EB985475EA98280C207C18312
:100F50005EB5C5B71A31FD77FD17F98F1EB103587D
:100F6000050256215E2D6577D2211307F7CF7D8FBD
:100F7000F9772206FD17518FB3F70701F22103D845
:100F8000A500C2064207336606013206D18F373606
:100F90000140C207130606C0C1824183C183631AA0
:100FA000C50071767D16F18EF2251A06D18EC20625
:100FB000C18256A1B71600405AAD9386068098416B
:100FC0006315D50038C11EB1828042074183DDBF61
:100FD0001E2189C593E717001EA18280C207C18325
:100FE000F99BC207C183CDBF8357450491C52167D3
:100FF000D98F2312F5048280C607C583DDBF5E2525
:1010000001C6DD8D4EA5828093C5F5FFFD8DDDBF48
:101010001E2189C593E707081EA18280C207C183EC
:1010200093F7F7F7C207C183C5BF5A2DFD779387A2
:10103000F77FF98FA205CD8FC207C1835EAD828095
:10104000B7170040938707806314F5002CC1828096
:10105000C205C181E5BFB7170040938707806314BD
:10106000F500485182804A314205418182801E2923
:101070004A25ED8F4205418189C76D8D3335A0002A
:1010800082800145828093C5F5FFC205C1810EA90A
:101090008280EFF2EF8D1629F577FD17F58FF62197
:1010A000DA257971D58F1EA95625FD779387379F4D
:1010B000F58FD6212A842EC6D58F9625D58FB625B5
:1010C000D58F5EA55E29C207C18393F7F7CFD98F6D
:1010D0005EA96808B539B747014093870780B245D4
:1010E000631AF404A25756246547B387E702C20681
:1010F000C186984163D20604060752244206B3D73C
:10110000E702130740064186B3D6E702B3F7E702CA
:101110009206635506028E0793872703B3D7E7022B
:1011200013F77700B367D700C207C1831EA44561D8
:101130006FF04F86925745BF0A07C1B79207938752
:101140002703B3D7E702BD8BD58FF9BF91C55E25C5
:101150000967D98F5EA582805A25F977FD17F98F27
:10116000D5BF13F7F50F85471583B395B7006319FE
:10117000F7009307C500984301CED98D8CC38280B8
:10118000894693074501E318D7FE93070501E5B7A4
:1011900093C5F5FFF98DDDB793F5F51F4EA182805C
:1011A0004A211375F51F82800A216D8D3335A00009
:1011B000828013F7F50F85461583B397B600631148
:1011C000D7025A25F98F1A2101454207418381CB65
:1011D0000545A181B315B5006D8F3335E0008280E0
:1011E00089466314D7001A29F1BF5A29E1BFEFE2FB
:1011F0003FF879711306000281450808EFE05FFAB5
:101200008545114502C202C402C631398545130520
:101210000020113901451D36371501409307E00FB5
:101220004C0013050580372401407C8202C6EFF094
:10123000AFEE13050440EFF06FA913050440EFF083
:10124000EFC6AA85239AA18237850000130545477A
:10125000EF50B02BB7070E003ECE0C0885471305A4
:1012600004402302F10202C802CA02CC02D0EFF00D
:101270006FA8854513050440EFF02FAD8545130594
:101280000440EFF08FC0814513050440EFF04FBDDF
:1012900013050440EFF06FAC930404402685EFF093
:1012A0006FAC6DFD1305044037240140EFF00FAC27
:1012B000930404402685EFF00FAC6DFD37050080E8
:1012C000B53C130504408545EFF00FBB93050002C4
:1012D00013050440EFF08FBC45616FE0BFEBEFE218
:1012E0003FE90111854521453D3E85451165993E02
:1012F0003714014085678D447C808A85C14713057A
:1013000004C03EC426C2EFF02FE1130504C085657A
:10131000EFF0CFED896761498A85130504C07C80B1
:101320004AC426C2EFF04FDF91677C808A859147DF
:10133000130504C03EC4EFF02FDEE1778A85130564
:1013400004C07C804AC426C2EFF00FDDB707040159
:101350003EC6B70702003EC8B707000285073744FC
:1013600000403ECAA1473ECC6C009D471305048057
:10137000FC863936854513050480253E05616FE0FE
:101380007FE1EFE25FDDB74400402A891304900C4F
:101390009389048089454E85353E0DC5CA851385E0
:1013A0000480B74400401D361304900C1389048058
:1013B00085454A85053611CD13850480113E137588
:1013C000F50F31A07D141374F40F69F401456FE03B
:1013D000DFDB7D141374F40F61FCCDBFEFE25FD946
:1013E0003714014001468565130504C0EFF04FE056
:1013F0001545413F1305F00F6937AA8405461305CB
:1014000004C08565EFF0CFDE26856FE0BFD8EFE240
:101410003FD6E937058975FD6FE0DFD7EFE25FD58D
:101420003714014001468565130504C0EFF04FDC19
:101430001945813F05468565130504C0EFF04FDB74
:101440006FE05FD5EFE2DFD21314C500B71401409F
:10145000F137753F01468565138504C0EFF04FD91C
:1014600013050002393F135504011375F50F113FA1
:10147000135584001375050F2937014519370546A3
:101480008565138504C0EFF0AFD651376FE09FD06C
:10149000EFE21FCE2A89371501402E84130505C0BF
:1014A0008565B2840146EFF0AFD40D45D93D1355A3
:1014B00004011375F50FF135135584001375F50FFD
:1014C000C9351375F40F753D014493170401C183A9
:1014D00063EC97003715014005468565130505C087
:1014E000EFF00FD16FE01FCB1305F00F593DB3079D
:1014F000890088A30504D1BFEFE29FC72E842A8903
:10150000B284293F3715014001468565130505C0A2
:10151000EFF00FCE0945B535135504011375F50FDE
:101520008D35135584001375F50FA13D1375F40F18
:10153000893D014493170401C18363ED970037157A
:10154000014005468565130505C0EFF06FCAC1353A
:101550006FE05FC4B3078900882305041D35D9BF38
:10156000EFE27FBF13F7F50F93070010998F3E84CA
:10157000C207C183AA892E89B2846373F6003284BC
:1015800042044180130A00102286CA854E85AD3779
:10159000638F8400818CC204C180A2992299268421
:1015A00063749A001304001042044180F1BF6FE09D
:1015B000DFBDEFE27FB913994501135949018567F2
:1015C000B38727413E84C207C183AA8AAE89B28409
:1015D00013DAC5006373F6003284370B002042042F
:1015E000930BCB214180130BCB21130CF00F931CD9
:1015F000CA000566E6855E85613D81471397070150
:101600004183636687002286CE85568525A8850797
:101610003307F9005A970347F7FFE30187FF528525
:10162000153581473387FA0014233307F9005E9795
:10163000850714A3139707014183E36587FE0566B9
:10164000E6855A85313F63838402A29AA299338446
:10165000844093140401C1808567050A01492684EA
:1016600063F3970005644204418051B76FE05FB1B6
:10167000EFE21FB0411185451145EFF0CFFA930716
:1016800000107C8237150140C1473EC64C008D4793
:10169000130505803EC4EFF02FA841016FE09FAF16
:1016A000EFE21FAD411185454145EFF0CFF785676A
:1016B000938707807C8237150140C1473EC64C00A6
:1016C0008D47130505803EC4EFF00FA541016FE083
:1016D0007FACEFE2FFA9411185452145EFF0AFF462
:1016E00093070010371401407C82C1473EC64C006E
:1016F0008D47130504C03EC4EFF00FA201469305C9
:101700000010130504C0EFF0AFAE41016FE09FA8D9
:10171000EFE21FA6797185452545EFF0CFF091479F
:1017200037150140FC824C0893078004130505C05F
:101730003ECEEFF06F9E89450545EFF0CFBE914755
:1017400005443ED00810B1473ED422D602D2EFF075
:101750008F93930780117C86680089475C8722C835
:10176000EFF08FD845616FE0FFA24111114522C60D
:10177000EFF00F9885476317F5022A841145EFF0C3
:101780000F9903C7618919EFB7450000371500208D
:1017900081461306803E9385C5EF1305052A238BEA
:1017A0008188B52B3244410173002030EFE25F9C09
:1017B000797185451545EFF00FE7856737150140CD
:1017C000FC824C0893078002130505803ECEEFF0A3
:1017D000AF94B1450145EFF00FB5856705443ED0A4
:1017E0000810A1473ED422D602D2EFF0CF8993074A
:1017F00080137C8668008D475C8722C8EFF0CFCECF
:1018000045616FE03F990565EFF08F8E8547631660
:10181000F5020565EFF0AF8F83C7C187B7450000BC
:1018200037150020850781461306803E938565F6AF
:1018300013050528238EF186DD2173002030EFE2A9
:101840003F93411185452145EFF0EFDD8545114579
:10185000EFF04FDF93070020371401407C82E1470F
:101860003EC64C008D47130504C03EC4EFF0CF8A3E
:10187000930700084C00130504C07C82EFF0CF8969
:1018800041016FE03F91EFE2BF8E01114D3F3714F0
:1018900000409307F01D8A85130504803EC002C2F4
:1018A0002314010023050100EFF06FE3130504800A
:1018B0008545EFF0EFF5C167938707066C001305C8
:1018C00004803EC8231B010002C6EFF0AFE81305F9
:1018D0000480A145EFF06FF5130504808545EFF016
:1018E0002FEF854513050480EFF00FF005616FE0E1
:1018F0007F8A411122C42A8408414AC24EC006C6CA
:10190000EF50400DB787000003A6874983A6C7495B
:101910002A89AE89EF30003B635F0502B78700007C
:1019200083A7C7481CC0B787000083A54749084064
:10193000EF40D003EF40706B931505013715004061
:10194000C18113050580EFF0AFEFB2402244124988
:10195000824941018280B787000003A6074A83A617
:10196000474A4A85CE85EF30002BE35EA0FAB78761
:10197000000083A707497DB7EFE28FFF7971371425
:101980000140C1472A89FC828D44C1474C08130598
:1019900004C03ECE26CCEFE03FF80146130504C05C
:1019A000C145EFF0EF8485452145EFF0CFC7854570
:1019B00037050800EFF00FC98547FC824C08E14766
:1019C000130504C026CC3ECEEFE01FF589449147B5
:1019D0004C08130504C0E482375400403ECEEFE0CB
:1019E000BFF30C10B7070C00130504C04AD03ED457
:1019F00002D223160102EFF0CFE99307D0137C86C1
:101A0000680085473EC84487EFF00FAE05461305D2
:101A100004C093055052EFF0CFF48545130504C080
:101A2000EFF0CFF245616FE0EFF6EFE26FF479711E
:101A300037140140930700022A89FC828D44C14774
:101A40004C08130504C03ECE26CCEFE0FFEC014667
:101A5000130504C093050002EFE09FF98545214579
:101A6000EFF06FBC854537050400EFF0AFBD93077D
:101A70000040FC824C08E147130504C026CC3ECE52
:101A8000EFE09FE9856793870780FC824C089147C8
:101A9000130504C03ECE37540040EFE0FFE70C10C2
:101AA000B7070C00130504804AD03ED402D2231697
:101AB0000102EFF00FDE930770137C8685475C8789
:101AC000680085473EC8EFF02FA205461305048045
:101AD00093055052EFF0EFE8854513050480EFF0D1
:101AE000EFE645616FE00FEBEFE28FE82A84EFF05D
:101AF000AFEA930500082285EFF00FEB7DD96FE088
:101B00006FE9411122C63754004093055052130526
:101B10000480EFF00FEA0DC513050480EFF04FE8E5
:101B20009375F50F238CB18203A5418A1C4D104992
:101B300054498507B3E7C7026384D70031055D24A4
:101B40003244410173002030411122C63754004015
:101B500093055052130504C0EFF0AFE50DC5130512
:101B600004C0EFF0EFE39375F50F238EB18203A568
:101B7000818A1C4D104954498507B3E7C702638425
:101B8000D700310585243244410173002030EFE253
:101B90002FDE0111AA842E8409458545EFF08FAA16
:101BA000E084370400404C081305044026CA231E75
:101BB0000100231D0100EFF08FB21305044085459D
:101BC000EFF06FCC0546854513050440EFF02FC3B9
:101BD0009307D0027C8685475C87680085473EC8AE
:101BE000EFF08F9005616FE0EFDAEFE26FD8B707A3
:101BF000002083A58716896793870771B3D5F502FF
:101C00007D1542054181FD15C205C18149376FE04F
:101C10006FD8411122C637040040854513050440A2
:101C2000EFF0EFC401C9854513050440EFF0AFC5DF
:101C3000EF00B0353244410173002030EFE24FD362
:101C400001112E84AA8485450545EFF0AF9F4C080D
:101C50003705004026CAE084231E0100231D010031
:101C6000EFF0EFA70546854537050040EFF02FB9A7
:101C70009307C0027C868D475C87680085473EC815
:101C8000EFF08F86854537050040EFF06FB40561B2
:101C90006FE04FD0EFE2CFCDB707002083A58716C6
:101CA000896793870771B3D5F502A9473305F50214
:101CB000FD15C205C1817D154205418141376FE0A7
:101CC0006FCD854537050040EFF06FBA19C58545E2
:101CD00037050040EFF02FBBD12873002030B7F755
:101CE00000E023A20700D92073002030411122C652
:101CF000373401408545130504C0EFF04FB701CDDF
:101D0000130504C08545EFF00FB8378500001305B3
:101D1000854AEF50C01032444101730020301DC984
:101D2000B296C206C18252A136A10CC509EE854702
:101D30001CA183A6018493870184368701EB54C5D7
:101D400088C30145828023000500E5B76306A7002C
:101D50005847EDB77D558280054582800DC583A724
:101D600001841387018499E305458280D4476396F3
:101D7000A6005845D8C7014582806394A70014C3C4
:101D8000DDBFB687CDB77D558280EFE26FBE03A47D
:101D9000018475DC1C2093F7F70F99C75E2099C367
:101DA000230004001C4482974044E5B783A70184C4
:101DB000054691E38280D62381CEBA237D17420760
:101DC0004183BAA3BA234207418319E390A3B6A380
:101DD000DC47C5B7232605000CC150C123240500EC
:101DE000054582805C45544118458507B3E7D70215
:101DF000638EE70058451C41BA978CA35C45584157
:101E00008507B3E7E7025CC5054582807955828086
:101E100018455C45630FF70018451C41BA979C2391
:101E20009CA11C4558418507B3E7E7021CC5054541
:101E30008280014582805C4518454841998FAA9768
:101E400033E5A7028280B707002083A787160967BA
:101E5000130707F4B3D7E702C207C1832393F184C2
:101E60002392F1848280B7F700E0D8438146799BC2
:101E7000D8C303D741843306A70290CBD4CB984371
:101E80001367070198C398431367170298C3D84391
:101E9000058B75DF9843799B98C38280EFE24FAD45
:101EA0002A841165011185451105EFE0DFF79307DD
:101EB00000207C82371501408D473EC44C00E1472D
:101EC000130505803EC6EFE03FA522C83744014018
:101ED000B70708000C08130504803ECC02CA231E75
:101EE0000100EFF00F9B854513050480EFF00FA66E
:101EF00005616FE02FAAEFE20FA6B7440140AE895B
:101F00003289014493840480634524014A856FE04B
:101F1000CFA7930500042685EFF00FA97DD9B387DD
:101F200089008385070026850504C205C181EFF07D
:101F3000AFA6D9BF138781801C43B71600209386B4
:101F400086523E95636BD500B75600209386068077
:101F500063E5A60008C33E858280FD57EDBF039769
:101F6000418381472A97634F070009CD0566930691
:101F7000F6FFB6876358C700AA876305D500931795
:101F80000701C1833E858280EFE2EF9C4111372437
:101F90000140AA8944001309010113040440CE85BD
:101FA000228595460546EFE00FDF85452285EFE067
:101FB0000FDD89452285EFE00FEA65DD2285EFE040
:101FC0000FE942054185613F8AA08904E31999FC24
:101FD0001547814735A013961700140885073696D4
:101FE000080893961700AA96835546FF03D546FF27
:101FF0006376B500231AA6FE239AB6FEC207C183F4
:10200000E3CBE7FC7D1771F728843C8541013E95C1
:102010004205418105816FE04F97EFE26F950545DD
:10202000A537EF40500EB787000083A5874BEF30F0
:10203000F051EF40301AB787000003A6074C83A683
:10204000474CEF209053B787000003A6874C83A628
:10205000C74CEF209052EF40B0226FE0AF93EFE219
:102060002F9109451537EF40100AB787000083A567
:10207000874BEF30B04DEF40F015B787000003A657
:10208000074C83A6474CEF20504FB787000003A6AC
:10209000874E83A6C74EEF20504EEF40701E6FE074
:1020A0006F8FEFE2EF8C0D45C535EF40D005B78758
:1020B000000083A5874BEF307049EF40B011B78720
:1020C000000003A6074C83A6474CEF20104BB787B0
:1020D000000003A6874C83A6C74CEF20104AEF40B0
:1020E000301A6FE02F8BEFE2AF881145713DEF4062
:1020F0009001B787000083A5874BEF303045EF4054
:10210000700DB787000003A6074C83A6474CEF204D
:10211000D046B787000003A6074E83A6474EEF20A0
:10212000D045EF40F0156FE0EF86EFE26F84194580
:10213000A13DA1679387074F01479306100F922394
:102140006369C5023A85EF30B002B787000003A685
:10215000074D83A6474DEF205042B787000003A6E6
:10216000874D83A6C74DEF30C00CEF4070116FE074
:102170006F8205078907E314D7FC13050000C5BF6C
:10218000EFD21FFF130620038145EFF08FC26FE0EF
:102190006F80EFD2FFFD397168001306200381457F
:1021A000EFF00FAF1886930730053705002063174F
:1021B000F70298869307C0046312F7020347D1031E
:1021C000D947631DF700130620036C0013050502B1
:1021D000EF409028054521616FD0DFFBB707002055
:1021E00003C74705130505029387470518A19833D0
:1021F00018B1B82338A1B83338B1D82358A1D8338F
:1022000058B1F82378A1F83378B19827DC3718A5AE
:10221000A308F5020145C1B7EFD29FF539712A84B1
:102220001306200381456800EFF08FA618869307F8
:1022300030056316F70298869307C0046311F7020E
:102240000347D103D947631CF700130620036C0032
:102250002285EF407020054521616FD0BFF3B7079D
:10226000002003C7470593874705014518A0983309
:1022700018B0B82338A0B83338B0D82358A0D83312
:1022800058B0F82378A0F83378B0982718A4DC3732
:10229000A308F402D1B7EFD21FECB7170020938741
:1022A000C721F82FC03FAA852207418FE03F13893D
:1022B000C1804204418F03C407026204598C228505
:1022C000EF400014B787000083A50772EF30106A53
:1022D000B787000083A58771AA892285EF3010692E
:1022E000AA854E85EF30E06F83250900EF30606FDF
:1022F0002320A9001385C180EFF0AFDF6FD0FFE886
:10230000EFD27FE5B71700209387C721F827C037A2
:102310002207418FE0371389C1804204418F802B0F
:102320006204598CA285EF40A00DB787000083A5F9
:102330000772EF30B063B787000083A58771AA8961
:102340002285EF30B062AA854E85EF308069832503
:102350000900EF3000692320A9001385C180EFF048
:102360004FD96FD09FE2EFD21FDFB71700209387BE
:10237000C721F82BC03B2207418FE03B1389C18066
:102380004204418F802F6204598CA285EF404007A0
:10239000B787000083A50772EF30505DB787000054
:1023A00083A54771AA892285EF30505CAA854E85A6
:1023B000EF30206383250900EF30A0622320A900BD
:1023C0001385C180EFF0EFD26FD03FDCEFD25FDA40
:1023D000371400201307C4218347C7028346B7027E
:1023E0000947A207D58F6387E7086367F7000547AA
:1023F0006387E7026FD01FDA0D476384E708114750
:10240000E39AE7FE938421819C2013844185DDC3F8
:10241000B707002093870702A83FDC2FBDA81389C8
:102420000181834709001304C4219384018685C771
:10243000B707002093870702883FBC2FA2075D8D56
:10244000EF40604CB787000083A5876DEF30101018
:1024500088C0230009002C2C1C3C8840A205DD8D7F
:102460003C3CC207CD8F4C2CE205DD8DEF30605730
:10247000DD3D49B7B787000003A5C76DEFF0BFE1A9
:1024800095BF938411819C201384C18485C7B707AD
:10249000002093870702E83B9C2FA2075D8DEF4049
:1024A0008046B787000083A5876DEF30300A08C0EB
:1024B000238004000840EFF0BFE42DBFEFD2DFC857
:1024C0001389318183470900138AC185D1C7370435
:1024D0000020130404027C244834B7840000A207BF
:1024E0005D8DEF40404283A5846DEF30300623A41C
:1024F000A1841C286834A2075D8DEF40C04083A5ED
:10250000846DEF30B00423A8A1843C280838A207CA
:102510005D8DEF40403F83A5846DEF30300383A590
:10252000846D23ACA184EF307044EF40E025AA8590
:10253000378500001305856FEF40207D7C284838E3
:10254000A2075D8DEF40203C83A5846DEF30100025
:102550002320AA0023000900371400209307C42178
:10256000B82F03C9970183C9570122073367270191
:1025700003C9B701EC2F03250A0042093367E900BC
:1025800003C9C701A2051304C42162093369E90024
:10259000F82B22073367370183C97701C20933E774
:1025A000E90083C98701E209B3E9E900D83FD98D81
:1025B000F83F42074D8F83C50702E205D98DEF3002
:1025C000D0296353A006CE854A85EF301029635287
:1025D0000502CA854E85EF30B062EF40A03FB78755
:1025E000000003A6874983A6C749EF20A06D635D5D
:1025F0000502378500001305C570A30504022306F4
:102600000402EF40D001EF100018B7350000371575
:10261000002081461306803E9385E5691305053049
:10262000EFF0EFEF6FD0DFB5CA854E85EF30505D2C
:10263000EF40403AB787000003AB874983ABC749F7
:102640002A8A5A86DE86AE8AEF20C067635E05005E
:10265000CE854A85EF30D05AEF40C0375A86DE86A5
:10266000EF204066634E05023C280438A207C58F60
:102670002438C204C58F4428E204DD8CB7870000EB
:1026800083A5076E2685EF30501D634BA000B787EA
:10269000000083A5476E2685EF309024635A05001D
:1026A0009147A305F40223060402238F01869DBFF0
:1026B00003AC81842685EF40E0312A8B6285AE8BA6
:1026C00083AC0185378D0000EF40C03003268D6E4E
:1026D0008326CD6EEF1030615A86DE86EF20805E55
:1026E000635005046685EF40E02E03268D6E832639
:1026F000CD6EEF2010342A86AE865A85DE85EF2017
:10270000605C634FA000B787000003A6076F83A635
:10271000476F5285D685EF20005089476342A00657
:10272000E6852685EF3070136355A00403AB8185E1
:102730005A85EF40202AB787000003A6076F83A6BB
:10274000476FEF10505A2A86AE865285D685EF2005
:10275000804C8D4763560502CE855A85EF30F00FC9
:102760006359A000CA855A85EF30300F91476349FD
:10277000A000E2852685EF30B016E35505EA8547CF
:10278000A305F4022306040271BDEFD2FF9BEFF014
:10279000DF88B71400201384C4219357850048B8FC
:1027A0007CA89357050161817CB808ACEFF07F8F5E
:1027B0009357850008BC3CAC9357050161813CBC34
:1027C00048ACEFF0DF899357850048B47CA4935759
:1027D000050161817CB408A8EFF0FF909357850054
:1027E0007CAC935705017CBC3C2C034A940148BC4B
:1027F000A207B3E74701034AB40161812300A402A1
:10280000420AB367FA00034AC40193050000620A52
:10281000336AFA005285EF30807E0DE168285C381B
:102820009305000022055D8D7C38C207C98F082CF6
:1028300062055D8DEF30A07C6304050E7C28834A21
:102840005401D285A207B3E75701834A7401378B3D
:102850000000C20AB3E7FA00834A8401E20AB3EA3D
:10286000FA005685EF30D039AA8BEF40A0167C24B1
:10287000443403260B6FA207C58F643483264B6F45
:102880002A89C204C58F0428AE89E204DD8CEF20BA
:1028900080386359A00883A501885E85EF30100D4C
:1028A000AA852685EF30D035935785003CA89357ED
:1028B00005013CB803C7E18708B8618148A83E8498
:1028C00029EB832B4B6F032B0B6F4A85DE865A86D1
:1028D000CE85EF204034634EA000D6855285EF3080
:1028E0003032EF40200F5A86DE86EF20C03263522E
:1028F000A0022685EF40000EB787000003A687726E
:1029000083A6C772EF20003C635505008547238FDF
:10291000F18683C7718989E7EFF05FBAEFF01FABEB
:102920006FD01F86268549B7EFD29F843795000068
:102930001306F02285451305458EEF40003DB7177D
:1029400000209387C72103C5B70283C7C702A20728
:102950005D8D6FD03F84EFD2BF81379500001306A5
:102960003022854513050587EF40203AB717002030
:1029700003A547242181420541816FD0BF81EFD259
:102980002FFF379500001306702185451305858AB2
:10299000EF40A037B71700209387C721D85303C54E
:1029A0008702B797000083A5478A21836205598D66
:1029B000EF30C07BEF307063420541816FD08FFDF7
:1029C000EFD20FFB379500001306B02085451305A5
:1029D0000591EF408033B71700209387C7219853A4
:1029E00003C54702B797000083A5478A2183620584
:1029F000598DEF30A077EF30505F420541816FD0A5
:102A00006FF9EFD2EFF6379500001306F01F8545FA
:102A10001305C583EF40602FB71700209387C721A8
:102A2000984FC82FB797000083A5478A2183620576
:102A3000598DEF30A073EF30505B420541816FD06C
:102A40006FF5EFD2EFF2379500001306301F854582
:102A50001305C580EF40602BB71700209387C7216F
:102A6000D84B882FB797000083A5478A218362053A
:102A7000598DEF30A06FEF305057420541816FD034
:102A80006FF1EFD2EFEE378500001306701E85451B
:102A90001305857DEF406027B71700209387C72176
:102AA000984BC82BB797000083A5478A21836205FE
:102AB000598DEF30A06BEF305053420541816FD0FC
:102AC0006FEDEFD2EFEA378500002E841306F01485
:102AD000854513050573EF4040230547B7140020D3
:102AE000238CE1881385042B23820186EFF00FA746
:102AF0005C245834B7450000A20737150020D98F51
:102B00008146371700201306803E9385A5041305E0
:102B1000052E2388042A231EF720EFF04FA06FD044
:102B20006FE7EFD2EFE43714002023A4A188154704
:102B30000566B74500002386E18885448146130673
:102B400086BB938505DA1305042B23829186EFF06B
:102B50000F9D2308942A6FD0EFE3EFD26FE1D425C5
:102B6000DC35A206DD8E954763FDD7003785000072
:102B70001306401285451305C575EF4000196FD047
:102B80006FE1B425BC35A206DD8E9307002063FA01
:102B9000D700378500001306B01285451305C578A8
:102BA000E9BF378500001305457CEF404027C1BFD2
:102BB000C16769768146FD170506139706014183B3
:102BC0006364B7003E8582803307D5001823B98F30
:102BD000214713F81700858363050800B18FC207EA
:102BE000C1837D17420741836DF78506F9B7EFD2A0
:102BF0002FD83715004013050580EFE0CFC5EF4013
:102C0000C022EF4000289307100F3365F502A94753
:102C100029053305F5026FD0EFD7EFD2CFD303A745
:102C2000418A2A84BE84054693055052631CA7043A
:102C30003755004013050580EFE0AFD22285EF1035
:102C4000B009131905010945EFF0EFA12285EF1036
:102C5000B00883A7418A931905011359090193D933
:102C60000901014693055052375500406391870290
:102C700013050580EFE0EFCE330539413335A00071
:102C80006FD0AFD037550040130505C075B7130599
:102C900005C0CDB7EFD2CFCD370400208347040263
:102CA0004111130404025C801C3023150100AA8426
:102CB000DC803C20AD450A855C813C302316010058
:102CC000DC815C205C825C30DC827C205C837C303C
:102CD000DC831C245C84930710FDDC8485475C85C1
:102CE000EFF01FED93578500DC858347140348867A
:102CF000DC86EFF0DFEFEFF00F972685EFF0FFF1C6
:102D00006DF93D468A852685EF10E07283A7418ADA
:102D100005469305505237550040639997001305B7
:102D20000580EFE00FC441016FD0CFC6130505C089
:102D3000CDBFEFD2EFC33704002083470402411117
:102D4000130404025C801C3023150100AA84DC807B
:102D50003C20AD450A855C813C3023160100DC81B6
:102D60005C205C825C30DC827C205C837C30DC8399
:102D70001C245C84930700FDDC8485475C85EFF0B0
:102D80003FE393578500DC85834714034886DC8640
:102D9000EFF0FFE5EFF02F8D2685EFF01FE86DF9DE
:102DA0003D468A852685EF10006983A7418A05463E
:102DB00093055052375500406399970013050580DD
:102DC000EFE02FBA41016FD0EFBC130505C0CDBFB6
:102DD000EFD28FB703C9C500DC3501112209336971
:102DE000F90042091359094193140901C18095471B
:102DF00063FF970037850000A6861306500C8545B3
:102E00001305C575EF30707005616FD06FB7B425CD
:102E1000BC35A206DD8E9307002063FAD700378504
:102E200000001306B00C85451305C578E1BFAA89DB
:102E300002CA02CC231E0100930A4101368A370BD5
:102E40000020B307DA40C207C18363E5970C371A45
:102E500000201304CA241305C40013066002814530
:102E6000EFD00FB43707002083470702A3052401E2
:102E7000230504001CA0930707029433939A1400BF
:102E80001309070214B0B42334A0B43334B0D423EC
:102E900054A0D43354B0F42374A0F4339C2774B0FA
:102EA0001CA4930700031CB43714002081471304AB
:102EB000842563C5570993856400860593F5E50F5E
:102EC0001305CA24EFF0DFCE9317850021815D8DB5
:102ED0008347190356940AA03CA0EFF05FD1EFE0BE
:102EE0009FF84E85EFF07FD36DF913860A019305A5
:102EF000CA244E85EF10205483A7418A05469305C6
:102F0000505237550040639C370513050580EFE0AC
:102F10004FA5DDBD13044B09930B84031C4063993B
:102F200047015C40014536C68297B2462390AA000D
:102F30002104E3958BFE890A050A21B7101013F7C7
:102F4000E70F329713F61700B306F400035747FF55
:102F500011E22183850798A293F7F70F99BF130514
:102F600005C075B7EFD22F9F370400201304440625
:102F7000AA89AE84328A1309040398341C4063176B
:102F8000F7005C405286A6854E8582972104E316A1
:102F900024FF6FD08F9FEFD2AF9A41112A8CEF1090
:102FA000A04F630E052A5145EFE0FFEB37190020D3
:102FB0001306200381451305C9241304C924B70D42
:102FC0000020EFD0EF9D81498144014A930B14000A
:102FD000B79C0000379D0000138B0D026285EF1037
:102FE000A04F630E05266285EF10804C9307C9241D
:102FF000D2973EC688A3930A1A0089476384FA00D1
:1030000063820426182083C70D026318F710183056
:1030100083471B006313F710379500001306202722
:1030200085451305C594EF30504EA5476396FA06C3
:10303000B717002003D7C7218947631FF708382037
:1030400083472B00631DF708383083473B00631824
:10305000F708582083474B006313F708583083471D
:103060005B00631EF706782083476B006319F70641
:10307000783083477B006314F706182483478B005E
:10308000631FF704379500001306B0288545130524
:103090008597EF30904721A08547E3EB97F8A94744
:1030A0006385FA00894763F1970AB717002083D731
:1030B000C721094714346392E71213070003639989
:1030C000E606379500001306C02D85451305859D3E
:1030D000EF30B043C5498DA883C74186ADF383C7A0
:1030E000518195CB38303C20F98F5820F98F5830DA
:1030F000F98F7820F98F7830F98F1824F98F13071A
:10310000F00F639AE700379500001306002A854503
:103110001305459ABDBF91E085445286DE851305AF
:10312000C924EF30703393070003E3F947EB05AA96
:1031300041476398E602379500001306202E854527
:103140001305C59FEF30703C1834C1476312F70C6C
:10315000B54763FF570B8349D4008609C509568AD2
:10316000D9B7138706031377F70F0546636DE6009B
:10317000379500001306902E8545130505A2EF3004
:10318000D038B549D1B703C751811DCF1307000A05
:103190001306F02E6389E6041307100A6398E6000D
:1031A0001306502F854513054DA61DB7268763F3DB
:1031B000F40009479374F70F1306D02F8545138544
:1031C000CCA8EF30903491BF268763F3F400094711
:1031D0009374F70F13068030D5B79307000A639AEC
:1031E000F60013061031379500008545130505A438
:1031F00079B79307100A13067031E385F6FAA687AC
:1032000063F3E400894793F4F70F1306F0317DB7B9
:10321000E3973AF59385DAFF93F5F50F1305C92483
:10322000EFF01F99330744018347E7FF0347F7FF98
:10323000A207D98F6397A700B2479823D947630A9B
:10324000F7000D47A68763F3E4008D4793F4F70F6B
:10325000E9B556869305C9246285EFF0BFD04101D8
:103260006FC0DFF1A547E39CFAE2D9B3EFC2BFEE2E
:1032700003A5418AB79900005D710D469385C9B5D4
:10328000EF10601B1306000581450A85EFC05FF152
:10329000378A000003A5C1808325CA713714002036
:1032A0001304C421EF20906CEF30004EB79500005E
:1032B0002A86938505AB0A85EF30F04403A5418A41
:1032C000130600058A85EF100017130600058145D7
:1032D0000A85EFC0FFEC682C5C3C378900002205B2
:1032E0005D8D7C3C8325896DC207C98F034504022F
:1032F00062055D8DEF209067EF300049B7950000C3
:103300002A86938585AC0A85EF30F03F03A5418A74
:10331000130600058A85EF1000121306000581458B
:103320000A85EFC0FFE768245C348325896D220598
:103330005D8D7C34C207C98F082862055D8DEF2042
:10334000F062EF306044B79500002A86938545AE61
:103350000A85EF30503B03A5418A130600058A8594
:10336000EF10600D1306000581450A85EFC05FE38D
:1033700028281C388325896D22055D8D3C38C207BD
:10338000C98F482862055D8DEF20505EEF30C03F49
:10339000B79500002A86938585AF0A85EF30B03651
:1033A00003A5418A130600058A85EF10C00813069D
:1033B000000581450A85EFC0BFDE68285C3883259B
:1033C000896D22055D8D7C38C207C98F082C620586
:1033D0005D8DEF20B059EF30203BB79500002A8675
:1033E000938505B10A85EF30103203A5418A130693
:1033F00000058A85EF1020041306000581450A8523
:10340000EFC01FDA282C1C3C8325896D22055D8DB9
:103410003C3CC207C98F482C62055D8DEF201055DA
:10342000EF308036B79500002A86938545B20A852D
:10343000EF30702D03A5418A130600058A85EF0041
:10344000907F1306000581450A85EFC07FD50345AF
:103450006402834754023797000022055D8D83473D
:1034600074028325478AC207C98F03458402620517
:103470005D8DEF20B04FEF302031B79500002A86E8
:10348000938585B30A85EF30102803A5418A13067A
:1034900000058A85EF00307A1306000581450A850C
:1034A000EFC01FD003A501888325CA71EF20104CFF
:1034B000EF30802DB79500002A86938585B40A8564
:1034C000EF30702403A5418A130600058A85EF00BA
:1034D00090761306000581450A85EFC07FCC03C6B0
:1034E0004188B7950000938505B60A85EF30B02175
:1034F00003A5418A130600058A85EF00D0731306E1
:10350000000581450A85EFC0BFC98347A402034671
:103510009402B7950000A2075D8E9385C5B70A8512
:10352000EF30701E03A5418A130600058A85EF005F
:1035300090701306000581450A85EFC07FC603C65B
:10354000E187B7950000938505B90A85EF30B01B78
:1035500003A5418A130600058A85EF00D06D130686
:10356000000581450A85EFC0BFC303C66189B795D1
:103570000000938585BA0A85EF30F01803A5418ACB
:10358000130600058A85EF00106B130600058145C0
:103590000A85EFC0FFC003C6C187B79500009385B9
:1035A00005BC0A85EF30301603A5418A13060005D5
:1035B0008A85EF0050681306000581450A85EFC033
:1035C0003FBE8347C4020346B402B7950000A2077A
:1035D0005D8E9385C5BD0A85EF30F01203A5418A43
:1035E000130600058A85EF00106503A5418A0D4684
:1035F0009385C9B5EF0030649387D1879023371442
:10360000014093050010133616001305048090A3A3
:10361000EFD00FBE1387D1881C23850793F7F70FD0
:103620001CA329476399E70005469305001013057D
:1036300004C0EFD0EFBB61616FC03FB5EFC25FB3B5
:103640009387C1899843D566938606186307D70286
:10365000050798C3371401408564938504801305DA
:1036600004800546EFD0CFB801469385048013054A
:103670000480EFD0EFB76FC0FFB123A00700B707FA
:10368000EFBE37E700E0938707083CC7E1B7EFC21A
:103690003FAE03A5818AEFF01F906FC0BFAFEFC2AE
:1036A0003FADB704002093870402F42FD83FA20651
:1036B000D98E1387418110239384040293878186D6
:1036C00011C6230007001387D6FF9AA39A23050784
:1036D000420741836305D7009AA36FC0BFAB239015
:1036E000070037140020EFE01FA01304C421135774
:1036F00085002301E4029357850113570501A301B7
:10370000E402A300A4022302F402DC282A89A838D8
:10371000A2075D8DEF30201FB787000083A5876D5E
:10372000EF20C062AA854A85EF203013E357A0FA44
:10373000371500209304053013050530EFE00FE244
:103740002380040068245C343797000022055D8DD7
:103750007C34832587C4C207C98F082862055D8D24
:10376000EF20B00F3325A000238FA186B7450000BE
:1037700037150020814679469385A5B11305052F9D
:10378000EFE0EFD999BFEFC2BF9E37970000032744
:1037900007C53705004081451305054023A6E18094
:1037A000EFD01F8337150040814513050580EFD00A
:1037B0003F896FC03F9EEFC23F99138761863709EB
:1037C0000020130609021E23834606026C3E85076D
:1037D000C207A206C183CD8E6385F6001EA36FC00B
:1037E0003F9A2310070037140020EFE05F8793040F
:1037F000C42193578500C8B4FCA493570501618187
:10380000FCB488A8EFE07F8193578500C8B8FCA876
:10381000935705016181FCB888ACEFE09F8893570E
:10382000850088BCBCAC935705016181BCBCC8ACA9
:10383000EFE0BF8F93578500A382A4022383F40295
:10384000935705016181A383F4022384A402B71472
:10385000014093050010138504C0EFD08F98130921
:1038600009021304C421814701C99145138504C08D
:10387000EFD08F96B337A000A304F4027C2844381D
:1038800083499401A207C58F643823050402C2044A
:10389000C58F042CE204DD8C3C2C2685A207B3E7FF
:1038A00037018349B401C209B3E7F9008349C40170
:1038B000E209B3E9F900CE85EF209034AA8AEF300F
:1038C0006011B797000003A687C383A6C7C32A8BDE
:1038D000AE8BEF10203F635405047C24034AD400D0
:1038E0005685A207B3E74701034AF400420AB367CB
:1038F000FA00034A0401620A336AFA0083A50188C8
:10390000EF20D006AA855285EF20902F935785008F
:1039100008B83CA89357050161813CB848A883C703
:10392000E187138CE187C5EBB787000003AA076F17
:1039300083AA476F5A855286D686DE85EF10A02D62
:10394000634EA000A6854E85EF20902BEF308008B7
:103950005286D686EF10202C6352A00868245C346F
:1039600022055D8D7C34C207C98F082862055D8DF4
:10397000EF304006B787000003A6877283A6C772A0
:10398000EF104034635C050485472300FC00B797C3
:10399000000083A507C32685EF20206C6350A00498
:1039A00003C7418885476309F70003A5018893058C
:1039B0000000EF20C0641DE1B7450000371500206E
:1039C0009306800C1306800C9385E5C41305052926
:1039D000EFE0EFB421A00547E38BE7FAEFE0AFF0AB
:1039E000935785007CAC935705017CBC83476402E8
:1039F0008344540248BCA207C58F8344740261818A
:103A00002300A402C204C58F834484020345A90293
:103A1000E204DD8C8347990222055D8D0D05EF20C0
:103A20003062AA852685EF20A06B6358050283C605
:103A30007189094713847189639EE600B7450000C8
:103A400037150020814679469385A5B11305052FCA
:103A5000EFE0EFAC2300040059B30345890283472C
:103A6000790222055D8D0D05EF20905DAA852685E2
:103A7000EF20A05E635DA0028347690203455902FF
:103A8000A2075D8DEF20D05BAA852685EF204065DB
:103A9000635F0500B797000083A747C323A6F180A3
:103AA0001385C180EFD0FFE40547A38BE1888345F0
:103AB00064028347540203456902A205CD8F834502
:103AC0007402034484022205C205DD8D8347590236
:103AD00062044D8C5D8D0D05EF209056A285EF2080
:103AE0002060E35E05CE0947A38BE188EFF0BFC9F4
:103AF000FDB1EFC2EFE737050040854513050540EE
:103B0000EFD00FCDB71700209387C7210947A385B2
:103B1000E702238607026FC0EFE7EFC2CFE3138708
:103B2000E1881E238507C207C1831EA31147636C6A
:103B3000F700371500409305400613050580EFD0C8
:103B40002FD06FC08FE4130760041384E188138AB9
:103B50004187636BF70083290A0083A5C1804E85E6
:103B6000EF20A04F6351A00C371500201309052F3B
:103B70001305052FEFE08F9E930700001385C1808A
:103B80002320FA002300090023100400EFD07FD681
:103B900003C7E18785476315F700EFF09FF555B739
:103BA000930700001385C1802320FA00231004002E
:103BB000EFD03FD4EFE06FC62A84EFE08FCEAA8526
:103BC0002285EF20F003EF20F060B787000003A408
:103BD000076F83A4476F2286A686EF10C003E34ECB
:103BE000A0FAEFE00FCC2A89EFE02FC3AA854A851F
:103BF000EF201001EF20105E2286A686EF10A001B4
:103C0000E34DA0F8B7170020370500409387C72180
:103C10001147854513050540A385E7022386070262
:103C2000EFD00FBB39BF4E85EF20D05AB7970000B9
:103C300003A607C483A647C4EF00F00AEF20506430
:103C40002320AA0013854187EFD0BFCADDBDEFC294
:103C50008FD0138701891C233971850793F7F70FDC
:103C60001CA305476394E70237050040814513050F
:103C70000540EFD0EFB59305C0123715004013058E
:103C80000580EFD0EFBB21616FC02FD02D4763942B
:103C9000E702EFE08FB8AA84EFE0AFC0AA852685DF
:103CA000EF20007623A6A186EFE06FBB23A0A18AB8
:103CB0009305401AD9B75547E397E7FC371500201D
:103CC0009304052913050529EFE04F89238004009B
:103CD000EFE0AFB42A89EFE0CFBCAA854A85EF2098
:103CE00020729384018788C0EFE06FB7AA8503A58F
:103CF000018A13840189EF20A0702A898C4003A5D2
:103D0000C186EF20E06FAA854A85EF202004B7978F
:103D1000000083A5C7C2138901882320A900AA89AE
:103D2000EF20A03393840188634FA0004E85EF20DD
:103D3000704AB787000003A6874983A6C749EF00EA
:103D40007078635A0500930700009CC023000400AC
:103D5000EFF03FDA0DBF6800EFE00FCCB784000052
:103D600015C583A5C47103250900EF202040EF206D
:103D7000D02742054181A306A10221812307A10288
:103D80006800EFE0EFBF23820188C9B7B7050020C4
:103D900013062003938505026800EF20F06BD1B76E
:103DA000EFC26FBB138791891C2301119386170003
:103DB000F51714A393F7F70F9306B00F63E3F6021A
:103DC000371500201304052B1305052B23820186CC
:103DD00023000700EFD09FF82300040005616FC0A7
:103DE000CFBA414681451305E100EFC06FBB3704F0
:103DF00000208347040213040402DD455C821C306A
:103E0000480093849189DC82FD577C83FD573EC432
:103E1000E9779387F71F7C8683C7C188DC87B7174C
:103E2000002003C7D72183C6C7219387C721220754
:103E3000558FA308E1009356870038202308D1004E
:103E40002309E1003830A309E1005820230AE100EA
:103E50005830A30AE1007820230BE1007830A30B4F
:103E6000E1001824230CE1009837BC27A207D98F62
:103E700013D78700230DF100A30CE100EFE05FD31F
:103E800093578500A30DF10083471403230EA1006F
:103E90002944A30EF100EFE09FD5EFD0DFFC13899A
:103EA000818803250900EFE05FD721E593878189A9
:103EB000942305476397E6002380070023800400CE
:103EC00031BF032509006D464C00B52303270900C7
:103ED00083A7418A05469305505237550040631722
:103EE000F70013050580EFD0CFA7CDBD130505C0A2
:103EF000DDBF7D141374F40F59FCCDB51387118900
:103F00001C233706002013060602850793F7F70FD8
:103F10001CA38346C6028345B602A206CD8E6393D8
:103F2000D704EFC2EFA4371500201304052A1305A8
:103F3000052A23000700238B0188EFD03FE22300EE
:103F40000400371401409145130504C0EFC0DFA8F9
:103F500001E9014693050010130504C0EFC05FA9F5
:103F60006FC04FA38280EFC2AFA003C761898547AE
:103F7000138421899384C1876312F70237150020C7
:103F8000130905281305052823000400239A018836
:103F900023800400EFD09FDC230009009820854790
:103FA0006315F7001C2085071CA037090020930625
:103FB000090283C7E60203C6D6021420A207D18FE6
:103FC000130909026392F60223000400371500204A
:103FD000130405281305052823800400EFD01FD8FB
:103FE000230004006FC00F9B854763FDE700371572
:103FF0000140014693050010130505C0EFC05F9F07
:10400000230004003715014093050010130505C077
:10401000EFC03F9D9387418901E59A2305079AA345
:10402000034709030346F90296232207518FE39BB6
:10403000E6FA37150140054693050010130505C043
:1040400023900700EFC0DF9A51B793878187904391
:10405000938651810506B705002090C32380060092
:104060009385050203C7450203C535022207498F20
:104070006314E602EFC2CF8F371500201304052E1C
:1040800023A007001305052E85479CA2EFD01FCD66
:10409000230004006FC00F908280EFC2CF8BB70463
:1040A00000209384040283C7240203C51402371935
:1040B0000020A2075D8DEF201005B787000083A5C3
:1040C000C7711304C921EF107048BC20938901887F
:1040D000370700203CA0BC3013074705230E0920FA
:1040E0003CB0DC20A30E092023A0A9005CA0DC309A
:1040F0001309C9215CB0FC207CA0FC307CB09C245E
:104100001CA43C271437A207D58F1CB4A1833CA460
:104110005C273437A207D58F3CB4A1835CA4EFD0D1
:104120001FF49357850048B47CA49357050161811F
:104130007CB408A8EFD07FEE9357850048B87CA8E0
:104140009357050161817CB808ACEFD09FF5935778
:1041500085015CAC7C24443413578500A207C58FCD
:10416000643438AC13570501C204C58F042838BC29
:104170005838E204DD8C7C28AA8508BCA2075D8F34
:104180007C38C207D98F182C62073365F700EF20FF
:10419000202783A50900EF10707DAA852685EF20D2
:1041A00020269357850008B83CA8935705016181E4
:1041B0003CB848A8EFD03FF393578500A300A40272
:1041C0002301F402935705016181A301F402230244
:1041D000A402EFD09FF5935785002303F402935771
:1041E0000501A303F4023C280438A302A402A20799
:1041F000C58F243861812304A402C204C58F4428DA
:10420000E204DD8CB797000083A5C7C42685EF10B4
:10421000306D634B0500B797000083A587C42685E2
:10422000EF10B0636355A00005472382E188B714FF
:10423000014093050010138504C0EFC08FFA814739
:1042400001C99145138504C0EFC00FF9B337A00031
:10425000A304F90223050902A305090223060902A2
:104260006FB0BFF2EFB2DFF0EFD0BFF2EFF0FFE2DE
:10427000B73500003715002081461306803E938530
:10428000C5261305052DEFD09FA9B73500003715BA
:1042900000208146130640069385E5681305053125
:1042A000EFD0FFA7B735000037150020F9461306F9
:1042B000803E9385C56313050532EFD05FA6B73501
:1042C0000000371500209306803E1306803E93853C
:1042D000657B1305052CEFD09FA4B735000037157B
:1042E000002081461306803E9385E569130505305D
:1042F000EFD0FFA2EFD07FA96FB0DFE9EFB25FE7A9
:104300000545EFD03F998D28EFD0EFD7EFC03FEEB6
:10431000EFD00FB6EFD0CFB8EFC07FFCEFD06FBBC0
:10432000EFD00FBFEFD08FC82945EFD01F8C6FB0F3
:104330007FE6EFB2FFE3014405C1002111CC5C41EF
:104340000D47639EE7003755004093F5F50F1305C1
:104350000580EFD06FF9054422856FB0BFE31147A8
:104360000544E39BE7FE3755004093F5F50F130531
:1043700005C0EFD06FF7CDB7EFB29FDF3704002055
:104380001304C40CB71500201306800C9385053365
:104390001305C400EFD01FA4716513050520EFD0ED
:1043A000CFE88544B715002004A01306C0129385FA
:1043B000853F1305840223A2818AEFD0BFA1485014
:1043C0007104EFD06FDB04A0014523A4818A6FB094
:1043D0007FDCEFB2FFD93715014005469305000297
:1043E000130505C0EFC0CFE06FB0DFDAEFB25FD8E2
:1043F00037150140014693050002130505C0EFC0C3
:104400002FDF6FB03FD9EFB2BFD637150140054659
:10441000C145130505C0EFC0AFDD6FB0BFD7EFB228
:104420003FD5371501400146C145130505C0EFC012
:104430002FDC6FB03FD6EFB21FD203A7418A2A8488
:104440002E8AB2899384418A6311A702EFF07FF824
:104450000149634339030545EFD0FFA09C406396B3
:104460008702EFF0BFF86FB05FD283A7818AE39134
:10447000A7FEEFF05FF9E9BFB3072A0183850700C4
:1044800022850509EFF0FFEAE9B783A7818AE39C5B
:1044900087FCEFF0DFF8C1BF814709C918218147C8
:1044A00011C75C49084D898FB337F0003E85828083
:1044B000EFB21FCC41112A84A3070100EFF0DFFD0A
:1044C00019C59305F1001305C400EFD07F940305CF
:1044D000F10041016FB01FCCEFB29FC93105EFD0A1
:1044E0009F956FB03FCB3708100001117D183377CF
:1044F000B80026CA3378D80093D4450113D34601B7
:10450000131E37004EC61357D5010E089357D60118
:1045100093F4F47F1373F37F06CE22CC4AC893D969
:10452000F50193DEF6013367C701131F350033E849
:104530000701931F3600338E64406380D919635698
:10454000C0136304031CB70680009307F07F336831
:10455000D800638FF4369307800363C0C735FD47E7
:1045600063CDC747130500023305C541B3D7CF015B
:10457000B316A8003399AF00DD8E33392001B3574D
:10458000C80133E926011D8F33092F41B3372F01AD
:104590003306F7409317860063D40724370780005B
:1045A0007D173374E600630C042C2285EF20E06352
:1045B000130785FF93070002998FB357F90033164D
:1045C000E400D18F3319E9006341972A33059740FE
:1045D000130615007D47634DC73813070002118F7E
:1045E000B356C9003319E9003397E700558F3339C3
:1045F00020013369270133D6C700814493777900BE
:1046000081CF1377F90091476308F700130749003A
:10461000333927014A963A899317860063D6071CD7
:10462000138514009307F07FCE856304F520B70748
:1046300080FFFD17F18F9398D70113593900A60712
:10464000B3E82801B1831375F57F9396C70052052F
:10465000F2406244B182FE05C98ECD8ED2444249F9
:10466000B2494685B68505618280631E0E0A1383B2
:1046700014001373E37F63170322B367E701B36882
:10468000F801639D041A6387074063860844330971
:10469000FF41B307074133362F013386C7409317D5
:1046A000860063D6074C3389EF41B307E84033B641
:1046B0002F013386C740F68991B76350C00F63005E
:1046C000030CB70680009307F07F3368D800638A35
:1046D000F43A9307800363CBC713FD4763DFC73505
:1046E00013090EFE93070002B3562801630AFE0069
:1046F000130900043309C94133192801B3EF2F010D
:104700003339F0013369D90031A2B367F801638A04
:10471000071C9307FEFF638C07389306F07F63093D
:10472000DE1A3E8E0DBDB305934063910422B3673C
:10473000E701638707329387F5FF63810744930698
:10474000F07F638CD520BE859307800363CCB72AA6
:10475000FD4763CFB73C930700028D8F3319F700F5
:10476000B356BF00B317FF003369D900B337F00069
:104770003357B7003369F9003308E84041ACB367F9
:10478000F801638007349307FEFF638A07209306CE
:10479000F07F6308DE2E3E8E2DBF631E0E149386BF
:1047A000140093F7E67F63910734B367E7016395DD
:1047B000042C6380073EB367F801638E073033092A
:1047C000FF01B3070701333FE9013386E701931780
:1047D000860063D70700B70780FFFD177D8E8544ED
:1047E00093777900E39F07E09317D6019358390038
:1047F000B3E8F800935736001307F07F638DE404A5
:10480000B207B18313F5F47FCE8581B53369F80122
:10481000333920017A99B337E9013386E7009317DA
:104820008600E3DF07FA85049307F07F6396F418A8
:10483000CE851305F07F8147814801BDC1EB6384BC
:10484000083A931636009317D8018D82B3E8D70043
:10485000F68993573800B3E7F800F9DB8145130573
:10486000F07FB70708008148CDB3370680FF7D167B
:104870007D8E93777900998CE39507D8B5B74A85F3
:10488000EF20A03613078501FD47E3D5E7D21306D5
:1048900085FFB317C900014905BB3369F8013339F6
:1048A0002001DDB13309FF413306074133342F01C5
:1048B000330486409317840063CD0724B3688900CE
:1048C000E39308CE8147814981441DBFE39808F8EE
:1048D0000E059317D7010D81B3E8A7009357370052
:1048E0009DBF0E059317D7010D81B3E8A700F28491
:1048F0009357370011B73305934063820412B7060C
:1049000080009307F07F558F630DF32E930780038C
:1049100063CBA720FD4763C3A72A93070002898FB3
:104920003319F700B356AF00B317FF003369D9004E
:10493000B337F0003357A7003369F9003A987E99EE
:10494000B337F901338607019A84D1BDB7068000D9
:104950009307F07F558FE319F3DE931736008D83AD
:104960009318D801B3E81701F68993573800E5B5D5
:10497000130715FE9306000233D7E700630AD6003B
:10498000930600043386C6403396C7003369C900D6
:10499000333920013369E9000146814491B5330977
:1049A000FF01B30707013336E9013E9693178600EE
:1049B0008544E3D707E28944B70780FFFD17F18FED
:1049C0001357190013791900336927019398F701D8
:1049D00033E9280113D6170015B113090EFE93070A
:1049E0000002B3562801630AFE00130900043309CC
:1049F000C94133192801B3EF2F013339F00133696D
:104A0000D90059B63369E7013339200133892F4181
:104A1000B3B72F013306F8409A84F689A5BEB36771
:104A2000E701638207189307F5FF6384071C930669
:104A3000F07F6304D5123E85D1BD93070002B38792
:104A4000C741B316F8003399FF0033D6CF01D18E9A
:104A500033392001B357C80133E926013E975DBBC6
:104A6000931736008D839318D801B3E81701AE84ED
:104A700093573800F68949B3EDC33369F801E31F52
:104A800009DC0E059317D7010D81B368F500935724
:104A90003700D1B36381080E931636009317D801FF
:104AA0008D82B3E8D700F6899357380091BB33095C
:104AB000FF41B3070741333F2F013386E741854468
:104AC000D1BC0E059317D7010D81B368F500F284B0
:104AD0009357370015B30E059317D7010D81B3E82F
:104AE000A7009357370029BB9307F07FE382F6D4E2
:104AF0003309FF013336E901B3070701B2979398F1
:104B0000F7011359190033E9280113D61700B684A9
:104B1000C1B93389EF413307E84033B62F0133047D
:104B2000C740F68949B43369E7013339200101BD33
:104B3000938705FE93060002B357F700638AD500FA
:104B400093060004B385B6403317B700336FEF0008
:104B50003339E0013369F90055BD931736008D8371
:104B60009318D801B3E8170193573800EDB1B36833
:104B7000C900E39708C68147814959B13389EF419C
:104B8000B307E84033B62F013386C740F689854422
:104B900011B4931636009317D8018D82B3E8D7006D
:104BA00093573800B1B9931636009317D8018D8208
:104BB000B3E8D700AA84935738003DB9930705FEA0
:104BC00093060002B357F700630AD500930600046A
:104BD0003385A6403317A700336FEF003339E00168
:104BE0003369F900A9BB81451305F07FB7070800B9
:104BF000A9BC3309FF01B30707013336F9013E961B
:104C000075B3931636009317D8018D82B3E8D70099
:104C10009357380089B113D74501B7071000FD1726
:104C200013D846011377F77F9308F07F33F3B7006B
:104C30002A8EF58FFD81B28E1378F87FFD8263088E
:104C40001703630018030DEBB368A3006314080097
:104C50005D8E29CA638508046388D502054595EDF4
:104C60008280B3E8C700E38008FE7955828033650F
:104C7000A30065FD630CE802631408005D8E79DE15
:104C8000E39ED5FCE34CE8FC63480701E3E867FCDE
:104C90006303F302637FF30081E57D558280F5DED7
:104CA000054582800145E39B08FA82805D8E69DAC2
:104CB0006DBF01458280E3E3CEFB0145E372DEFB7D
:104CC000E5F1E1BF13D74501B7071000FD1713D871
:104CD00046011377F77F9308F07F33FEB700AA8E63
:104CE000F58FFD81328F1378F87FFD82630E1703F5
:104CF000630D180129E3B368AE00631F08005D8EE1
:104D000001EE0143638C080421A8B3E8C7000943FE
:104D1000639608046DD305A0638408046385D502F7
:104D200005438DCD7D531DA8B368AE00094363973D
:104D30000802630AE802631408005D8E75D2E391ED
:104D4000D5FEE34FE8FC63490701E3EBC7FD630FC2
:104D5000FE0001436374FE00F1D505431A8582808D
:104D6000EDFE7D53E5BF5D8E79DACDBFE36ADFFBF3
:104D70000143E3F5EEFFF5F175B739714AD813D960
:104D800045014ED652D456D29399C50006DE22DC98
:104D900026DA5AD05ECE1379F97F2A8A93D9C900D0
:104DA00093DAF501630D090E9307F07F6306F91896
:104DB0001354D5018E09B36934013704800033E4FC
:104DC000890093143500130919C08149814B13D709
:104DD0004601139AC6001377F77FB285135ACA00AB
:104DE00013DBF601630B07109307F07F6303F704EF
:104DF0009357D6010E0A33EA4701130717C0B707C6
:104E00008000B367FA00931536003A99814833C79A
:104E10006A01BD463A851308190063E8361717463C
:104E20000000130666E38A09B29983A60900B296C8
:104E30008286B367CA001309F97F6399071293E961
:104E4000290081458948E1B701479307F07F37047E
:104E5000080081443204D20731807E075D8C598C72
:104E6000A285F250625426854259D254B259225A30
:104E7000925A025BF24B216182805A853E84AE8455
:104E8000C68B8947638DFB0E8D47E38FFBFA854701
:104E90002A87639EFB3881470144814465BF33E420
:104EA000A90061C036C632C4638C092A4E85EF1052
:104EB000D0532246B246AA87130755FF7544938400
:104EC00087FF198CB399990033548A0033643401F5
:104ED000B3149A0013D746011309D0C0139AC60021
:104EE0001377F77F3309F9408149814BB285135A13
:104EF000CA0013DBF601E31907EEB367CA00B1C7B6
:104F0000630F0A22528532C4EF10304E22462A87A0
:104F1000930655FFF547930587FF958F331ABA001F
:104F2000B357F600B3E74701B315B6003309E940BC
:104F30001309D9C08148E1BD33E4A90001ECA149BE
:104F400081441309F07F894B59B593E919008145D4
:104F5000854875BD4E84AA84B1491309F07F8D4BF5
:104F6000BDB5914981440149854B95B593E9390017
:104F7000D2878D4869BD89475685E397FBF02A871C
:104F80009307F07F01448144F1B5C16E1386FEFFA3
:104F900093D6040113DE0501F18CF18D3386950261
:104FA0003383B6029358060133059E021A95AA98D8
:104FB000B382C60363F36800F692C16F1383FFFFE9
:104FC00033F5670093D30701B3F76800C207337363
:104FD00066003E933306950293D80801B387A60274
:104FE000135F0601B3849302BE94FA94B38E7602E3
:104FF00063F3F400FE9E416A9307FAFF935F040196
:10500000B376F400B3F9F4007D8EC1803384D50209
:10501000C209338FD401B299CE98B307DE02935EF2
:105020000401B385BF02AE97BE9E330EFE0363F349
:10503000BE00529EC1679385F7FF33F6BE006D8CAC
:105040004206229693DE0E01B305D502769E338585
:10505000AF0213D40501B386D302AA96A296B38FEA
:10506000F30363F3A600BE9F41657D15B3F7A60069
:10507000C2076D8DAA97B3855800B3B93501FA9769
:10508000B2953384370133B6C500B30EC4013385FE
:10509000CE0033343401B3B7E701C18F33BECE0144
:1050A00013D406013336C5003E943366CE00939484
:1050B000950032947E94B3E46400260493567501FF
:1050C000B3349000DD8193179500CD8C558CDD8C29
:1050D0009317740063DB070093D714008588931639
:1050E000F401DD8CD58C058042899307F93F635923
:1050F000F00893F6740081CE93F6F40011466388AD
:10510000C60093864400B3B496002694B6849316E2
:10511000740063D80600B70700FFFD177D8C930766
:1051200009409306E07F63CFF60E93D634009314C4
:10513000D4012604D58C318093F7F77F21BB3285CB
:1051400032C4EF10902A93065501F1471307050268
:105150002246E3D1D7DC6115B317A6008145F9B328
:10516000EF10B02813075501F145930705022246B9
:10517000B246E3D5E5D461153314AA00814499BB46
:1051800085469D8EB1E71309E941B3972401B3D455
:10519000D40033192401B337F000B3649900DD8CD7
:1051A00093F77400B356D40081CF93F7F4001146FF
:1051B0006388C70093874400B3B49700A696BE8463
:1051C0009397860063D8070485470144814459B109
:1051D00013068003E341D6CC7D46E356D6FA055646
:1051E000B307F640930500023356F4006387B60018
:1051F0001309E943B3172401DD8CB3349000D18C3B
:1052000093F67400014499CA93F7F400114681465D
:10521000E392C7FA139496003180F6068D80D58C00
:1052200081470DB99307F07F0144814425B142893C
:105230006DBD370710007D1701113373B70093D888
:105240004601758F935ED60122CC26CA0E0393D4F5
:1052500045019357D5010E0706CE4AC84EC693F8AE
:10526000F87F130EF07F33E7EE0093F4F47F13D44E
:10527000F50133E36700131F3500FD82931E3600EE
:105280006380C81993C61600B38514416305D41210
:105290006351B018638B081AB70780005D8F638174
:1052A000C4599307800363C4B734FD4763C5B74847
:1052B000930700028D8FB3D9BE003318F700B39E59
:1052C000FE00336838013357B700B339D001336873
:1052D00038013303E340B3090F41B3373F013306CD
:1052E000F3409317860063D30724370980007D19A4
:1052F00033792601630F092C4A85EF10100F13072D
:1053000085FF93070002998FB3D7F9003316E900A0
:10531000D18FB399E9006344972A058F13061700CC
:10532000FD4663C5C63A13070002118FB3D6C90004
:105330003398E9003397E700558F33380001B3699C
:10534000070133D6C700814493F7790081CF93F6E4
:10535000F90091476388F6009386490033B8360117
:105360004296B6899317860063D6071C13871400EC
:105370009307F07F05886306F720B70780FFFD17C6
:10538000F18F1398D70193D93900A60733683801F4
:10539000B1831377F77F9396C7005207B1827E04DB
:1053A000D98EC18EF2406244D2444249B24942850C
:1053B000B685056182806356B00A638A0812B70712
:1053C00080005D8F6387C42D9307800363C7B71880
:1053D000FD4763D2B73C138805FE93070002B3591B
:1053E0000701638AF50093070004B385B7403317BC
:1053F000B700B3EEEE003338D0013368380195A220
:10540000B367D7019385148099E393C61600630AA6
:10541000D404D1E19387140093F7E77F6399071EC3
:10542000B367E3013368D701639204166382073CD4
:1054300063160842131835009316D3011358380029
:1054400033E806019357330019A2B367D701638588
:10545000071A9387F5FF638B073A638CC523BE85D4
:1054600089B56399051C9386140093F7E67FC1EF15
:10547000B367E30163900436638D0744B367D701D4
:10548000639407460E051318D3010D813368A800F5
:10549000935733006DA8B385984063970420B36792
:1054A000E301638D07309387F5FF63890740130598
:1054B000F07F6383A520BE859307800363C2B72A6C
:1054C000FD4763C8B73C930700028D8F3318F30084
:1054D0003356BF00B317FF003368C800B339F0007C
:1054E0003353B3003368380133076740B5ACB36753
:1054F000D701638307109387F5FF638F071E6380CF
:10550000C52FBE85D1B59307F07F638BF606FA9E53
:1055100033B6EE01B307E300B2971398F70193DEB9
:105520001E00B369D80113D61700B68493F779002B
:10553000E39F07E09317D60113D839003368F800CA
:10554000A685935736001307F07F6380E506B20700
:10555000B18313F7F57F05883DBD3367D701333835
:10556000E000B309E801B3B7E90133866700931798
:105570008600E3DD07FA85049307F07F639CF41847
:1055800005881307F07F8147014831B56391071003
:105590006301083C131836009317D70113583800DD
:1055A0003368F800368493573700B367F800E9DBB7
:1055B00001441307F07FB70708000148E9BB37062D
:1055C00080FF7D167D8E93F77900998CE39107D843
:1055D00095B74E85EF10606113078501FD47E3D253
:1055E000E7D2130685FFB397C90081492DB333680D
:1055F000D70133380001C5B1131835009317D30113
:10560000135838003368F800935733002DBFB3099F
:10561000DF413309E34033363F013309C940931773
:10562000890063CA072033E82901E31508CC8147C4
:10563000014431BFB385984063810414B7068000EC
:105640009307F07F3363D3006381F82093078003CF
:1056500063CCB722FD4763C9B72C930700028D8F37
:105660003318F300B356BF00B317FF003368D800F8
:10567000B339F0003353B300336838011A97B309D4
:10568000D801B3B7D9013386E700C684CDB5E3119D
:1056900008F2131835009317D301135838003368F4
:1056A000F8009357330011B7370580009307F07F58
:1056B0003363A300E392F8E00E061318D7010D82BE
:1056C0003368C800935737003684C5B5051793066D
:1056D000000233D7E700630AD6009306000433863E
:1056E000C6403396C700B3E9C90033383001B36907
:1056F000E800014681441DBDB309DF01B307E300A3
:1057000033BFE9013386E701931786008544E3DF61
:1057100007E08944B70780FFFD17F18F13D7190001
:1057200013F81900336807019399F701B3E90901E8
:1057300013D6170011B9138805FE93070002B35959
:105740000701638AF50093070004B385B740331758
:10575000B700B3EEEE003338D00133683801A5BE90
:105760003363E30133386000B3890E41B3B73E01C0
:105770003306F740C6843684ADB6B367E30163876A
:1057800007189387F5FF638C071C9306F07F638EE1
:10579000D50ABE8565BD930700028D8FB3D9BE00C3
:1057A0003318F700B39EFE00336838013357B70053
:1057B000B339D001336838013A9365B31318360012
:1057C0009317D7011358380033E8070136849357ED
:1057D000370095BBBDCB3367D701E31B07DC0E0554
:1057E0001318D3010D813368A8009357330075BB9C
:1057F000E30F08E2131836009317D7011358380047
:105800003368F80036849357370091B3B309DF410A
:10581000B307E340333F3F013386E7418544D1B4CA
:10582000131835009316D3011358380033E80601D6
:10583000935733009DBBB389EE413306674033B9BC
:105840003E0133092641368475B40E061318D7017C
:105850000D823368C8009357370081BBB309DF411D
:10586000B307E34033363F013386C74093178600C2
:1058700063D7070AB389EE41B3076740B3BE3E0161
:105880003386D7413684C9B43363E30133386000CB
:10589000FDB3138805FE93070002B3590301638A21
:1058A000F50093070004B385B7403313B300336F9B
:1058B0006F003338E001336838017DB5B389EE41BC
:1058C000B3076740B3BE3E013386D7413684854473
:1058D00009BC131836009317D701135838003368E2
:1058E000F80093573700A5B1B309DF01B307E30010
:1058F00033BFE9013386E70193178600E3D807C277
:10590000B70780FFFD177D8E85440DB10E06131875
:10591000D7010D823368C800935737002DB133E8A3
:10592000C900E30608D019B1138805FE93070002E9
:10593000B3590301638AF50093070004B385B740A8
:105940003313B300336F6F003338E001336838012D
:105950003DB301441307F07FB70708002DBCB3091E
:10596000DF01B307E300B3BED9013386D70169BBBA
:10597000411106C622C426C20DCD9357F541B3C4CA
:10598000A7009D8C2A842685EF1020269306E041EF
:10599000898EA9477D8093F6F67F63CDA7022D47B8
:1059A000098FB3D7E4005505B207B394A400B183BF
:1059B00029A00144814681478144B207D206B183C0
:1059C0007E04D58FC18FB24022442685BE85924485
:1059D000410182805515B397A400B207B183814479
:1059E000E9BF4111370780007D1713D8750126C222
:1059F000935475013373A70093F4F40FB376B70093
:105A00004AC01378F80F1359F50106C622C4FD8168
:105A10009A8726854A86131E3300939E3600B388E4
:105A20000441630AB90E6350100D63040814930710
:105A3000F00F638BF414B7070004B3EEFE00ED47DC
:105A400063C1172993070002B3871741B397FE007C
:105A5000B3D81E01B337F000B3E7F800B307FE4038
:105A600013975700635E0718370400047D147D8C7C
:105A70002285EF1080176D15B317A4006348951A9F
:105A8000058D1304150013070002018F3397E700FB
:105A90003337E000B3D78700D98F814413F77700FD
:105AA00019C713F7F70091466303D70091071397BF
:105AB0005700635B071485041307F00F4A8663835E
:105AC000E4169A07A58313F5F40FB2402244A60703
:105AD0009314750113D59700458D7E0692440249B3
:105AE000518D410182806399080A1387140013774E
:105AF000E70F6317071463900422630D0E1EE386FD
:105B00000EFCB307DE411397570063500722B3879B
:105B1000CE412E8961B7635C100B630E08089307B2
:105B2000F00F6383F406B7070004B3EEFE00ED4701
:105B300063C9171F93070002B3871741B397FE008D
:105B4000B3D81E01B337F000B3E7F800F29713970C
:105B500057006357070A85041307F00F6384E40CAA
:105B6000B706007E13D71700FD16858B758FD98F6A
:105B700035B7638D0E08FD18B307DE41E38208EEEA
:105B80009307F00FE39DF4EA630D03080146130544
:105B9000F00FB707400015BF33079840EDE86302E8
:105BA0000E147D17630807189307F00F6319F80E9A
:105BB0002E893683D1BF638B0E04FD18B307DE0137
:105BC000E38708F89307F00FE393F4F675BF639546
:105BD0000808850413F7E40F631307126317051011
:105BE000630F0E14E3830EEEB307DE011397570025
:105BF000814463570700370700FC7D17F98F854400
:105C000013F77700E31F07E813D337009307F00F6C
:105C1000E38CF4F693179300A58313F5F40F4A86EB
:105C20006DB54A861305F00F814745B5370700FC6F
:105C30007D17F98F13F77700898CE31407E6E9B72E
:105C40003304DE419317540063C3070CE31204E2EC
:105C500001460145814795BD33079840ADC4930780
:105C6000F00FE308F8F4B7070004336EFE00ED47C9
:105C700063CCE70C93070002998FB317FE003357EC
:105C8000EE00B337F000D98FF697C284C9B59307F9
:105C9000F00FE30FF8F0B7070004336EFE00ED4796
:105CA00063C3E70893060002998EB316DE00B3576C
:105CB000EE003337D000D98FB387FE40C2842E89DF
:105CC00045B3854761BB630E0E067D17B307DE0142
:105CD000C284E30E07E69307F00FE31AF8F8368361
:105CE00065B53683C2842E8915B7E3040EECE38DC7
:105CF0000EE869BD638D0E022E86B687F9B3930751
:105D0000F00FE381F4F2B307DE018583D5BD338460
:105D1000CE412E89B1BBE31C0EFCE3890EE62E8931
:105D200049BD854725B5854741BFE39B07EC014643
:105D3000814761BBB387CE41C2842E8915B3B68734
:105D400069B33683C284D9B585473DBF397193574E
:105D500075014AD856D25ECE931A95001359F501B3
:105D600006DE22DC26DA4ED652D45AD093F7F70F4D
:105D700093DA9A00CA8B638207121307F00F6384C9
:105D8000E7128E0A37070004B3EAEA00138A17F80D
:105D90000144014B93D775019394950093F7F70F46
:105DA000A58093D9F501FDC71307F00F6387E702BC
:105DB0008E04938717F837070004D98C330AFA400A
:105DC0008146558C17370000130707ED0A043A94F3
:105DD0001C4033493901BA978287130A1AF0F9E84F
:105DE0008946558C17370000130707EF0A043A94C9
:105DF0001C4033493901BA97828701491307F00FD4
:105E0000B707400013959700F2506254931777013B
:105E100025817E095D8D33652501D2544259B259E1
:105E2000225A925A025BF24B216182801307F00FD3
:105E30008147C9BFA68ACE8B368B8947630BFB1A75
:105E40008D47E30CFBFA8547630AFB0A1307FA0741
:105E500013F91B006357E01293F77A0099C793F781
:105E6000FA0091466383D700910A93974A0063D959
:105E70000700B70700F8FD17B3FAFA0013070A087E
:105E80009307E00FE3C4E7FA93976A00A5831377BB
:105E9000F70F8DBFB9E48546A9B763940A02114490
:105EA000014A054BC5BD63990A002144130AF00F4E
:105EB000094BCDB58D4631B73144130AF00F0D4B68
:105EC000D1BD56852EC6EF0050529307B5FFB39A49
:105ED000FA009307A0F8338AA7400144014BB2456A
:105EE00055BD2685EF0070501307B5FFB307AA0014
:105EF000B394E400138A67078146E1B513F91B00E8
:105F00000147814701B74166139554007D169357A9
:105F10000501698E63FA9A0AB3D5FA027D1AD6860C
:105F200001473388C502B3F6F602C206558F637B7C
:105F300007012A979386F5FF6368A70A6376070B24
:105F4000F9152A9733070741B356F7023377F7025B
:105F5000B38AC6029317070163FB5701AA971387F9
:105F6000F6FF63E1A70863FF5707F916AA97C20572
:105F7000B38A5741D58DB33A5001B3EA5501CA8B64
:105F8000F1B58546998E11C76D4601478147E34BB0
:105F9000D6E6130AEA09339A4A01B3D7DA00B33ACC
:105FA0004001B3E7570113F7770019C713F7F7005C
:105FB00091466303D7009107139757006348070280
:105FC0009A07A58301473DBD93D61A00B3D5F602C3
:105FD0001397FA0141833388C502B1B7CE8B368B54
:105FE000814AA1BDBA8661B7B685A9BF0547814779
:105FF00011BD13F91B001307F00F814721B593560C
:106000007501B7078000FD1713D6750193F6F60FDB
:106010001308F00FB3F8A7001357F501ED8F1376AF
:10602000F60FFD81638406031305F00F6304A602D7
:1060300005456383C6008280E39FF8FE0145E30CBB
:10604000B7FE0545EDFA3335100182800545E38D35
:1060500008FC82800545E9DF828093567501B70709
:106060008000FD1713D6750193F6F60F1308F00F95
:10607000B3F8A7001357F501ED8F1376F60FFD81E6
:1060800063810603630C06018DE211E2B1C3638EE6
:1060900008026305B70405451DE78280F5D77955E9
:1060A0008280E39E08FE6309D60211E2EDD7E31475
:1060B000B7FEE342D6FE63C7C600E3EE17FD014517
:1060C000E3FDF8FC01E77D558280F5DD0545828022
:1060D0000145E39208FC8280F9DBD1B78146E1BF3C
:1060E00093567501B7078000FD1713D6750193F617
:1060F000F60F1308F00FB3F8A7001357F501ED8F53
:106100001376F60FFD81638706036309060185EAAE
:1061100011EA89EB0145639B080082800945F5FF80
:10612000E5DA31A8638C08026300B704054575D72A
:106130007D5582800945639808026304D60211E206
:10614000F5D7E315B7FEE343D6FE63C7C600E3EF1A
:1061500017FD0145E3F3F8FC19E3D9BFF1D9054573
:106160008280E5D3828082808146C5B7797122D44E
:10617000135475014ECE52CC9319950006D626D2F3
:106180004AD056CA5AC81374F40F93D99900135AB7
:10619000F50169C49307F00F6308F40E9397390073
:1061A00037070004B3E9E700130414F88144014BF6
:1061B00013D77501939A95001377F70F93DA9A0026
:1061C00013D9F50145CF9307F00F630CF7028E0A40
:1061D000130717F8B7070004B3EAFA003A94014628
:1061E00033452A01BD47AA869305140063E2971040
:1061F00017370000130747B28A04BA949C40BA9735
:1062000082871304F40F63980A0C93E42400094670
:10621000C1BF01451307F00FB7074000B250225429
:10622000A6075E07A5837E05D98F92540259F249CD
:10623000624AD24A424B5D8D45618280CA86D689C8
:10624000328B89476301FB0A8D47E304FBFC8547DA
:1062500036856312FB1A01478147C9B7639E09045B
:1062600013D77501939A95001377F70F9144014462
:10627000054B93DA9A0013D9F50131F7639D0A00B3
:1062800093E414000546A9BF63930902A1441304D3
:10629000F00F094B31BF5685EF0030159307B5FF5E
:1062A000098CB39AFA001304A4F8014615BFB1444F
:1062B0001304F00F0D4BEDBD4E852EC6EF00F0120E
:1062C0009307B5FF1304A0F8B399F900098C814432
:1062D000014BB245F1BD93E434000D4611B7894737
:1062E000D286E313FBF636851307F00F81473DB7DF
:1062F00041639306F3FF13D6090193D80A01B3F75C
:10630000D900B3FADA0033885703B389F802135778
:106310000801B30A5603D6994E97330616036373E2
:1063200057011A96C167FD17B376F7003378F80066
:10633000C206C2969399660093570701B33930019C
:10634000E982B2979A07B3E6D900B3E9D7009397E9
:10635000490063D9070013D7190093F71900B369EF
:10636000F7002E841307F4076350E00493F77900D5
:1063700099C793F7F90091466383D70091099397E2
:10638000490063D90700B70700F8FD17B3F9F90012
:10639000130704089307E00F63CBE70493976900A2
:1063A000A5831377F70F9DBD8547B386E74011C7D7
:1063B0006D4601478147E343D6E61307E409339767
:1063C000E9003337E000B3D7D900D98F13F777004E
:1063D00019C713F7F70091466303D7009107139786
:1063E0005700634C07009A07A583014705BD1307B3
:1063F000F00F814725B52E84B5B70547814739BDD4
:106400003707800041117D179356750113D8750128
:10641000B377A70093F6F60F935EF5013376B700D6
:1064200026C24AC01378F80F06C622C41303F00F21
:106430003E8E3689F684139F3700FD811315360092
:10644000B38806416302681093C51500638CBE10C3
:106450006354100D631008106304051EFD18B30784
:10646000AF40638608029307F00F6388F616ED4786
:1064700063C7172913070002330717413317E500D5
:10648000B35715013337E000D98FB307FF40139797
:1064900057006351071A370400047D147D8C228550
:1064A000A9276D15B317A400634E251B330525419D
:1064B0001304150013070002018F3397E7003337E9
:1064C000E000B3D78700D98F014913F7770019C7C8
:1064D00013F7F70091466303D7009107139757000E
:1064E000635E0714930619001307F00F93FE140060
:1064F0006386E6169A07A58393F6F60FA607B240C1
:10650000224413D59700DE069397FE01558D9244E1
:1065100002495D8D410182806392080A138716004B
:106520001377E70F631B07146394062263020F209F
:1065300071D5B307AF401397570063550722B307D0
:10654000E5410149AE8451B7E30005F0638ABE0A14
:10655000E35410FD9307F00F6381F608B7070004BA
:106560005D8D31B7635E1009630108089307F00F72
:106570006385F606B70700045D8DED4763C0171FFE
:1065800013070002330717413317E500B35715010E
:106590003337E000D98FFA9713975700635C0708E9
:1065A00005091307F00F630BE90AB706007E13D73E
:1065B0001700FD16858B758FD98F01BF3307D84023
:1065C00063950610630D0F147D176303071A930775
:1065D000F00F6314F810AE84328E630F0E06814EF6
:1065E0009306F00FB707400011BF39C9FD18B30774
:1065F000AF00E38308FA9307F00FE390F6F8F1BFDA
:1066000063990808138916001377E90F63160712B8
:10661000639B061063030F16E30205EEB307AF009A
:1066200013975700014963570700370700FC7D1790
:10663000F98F054913F77700E31C07E813DE3700ED
:106640009307F00FE30BF9F893179E00A583937659
:10665000F90F93FE14005DB593FE14009306F00F3E
:10666000814769BD370700FC7D17F98F13F7770065
:106670003309A940E31E07E4D1B73304AF409317B1
:10668000540063C3070CE31C04E0814E814681473C
:10669000B5B53307D840B5C69307F00FE30EF8F24F
:1066A000B7070004336FFF00ED4763CDE70C930796
:1066B0000002998FB317FF003357EF00B337F00094
:1066C0005D8FB307A7004289C1BD9307F00FE304B4
:1066D000F8F0B7070004336FFF00ED4763C2E70827
:1066E00093070002998FB317FF003357EF00B337BA
:1066F000F000D98FB307F5404289AE8449BB854786
:1067000069B3630E0F067D17B307AF004289E30537
:1067100007E89307F00FE319F8F8328E7DBD328E4B
:106720004289AE8431BFE3090FEAE30805EA45BDBB
:106730000DCDAE8EB287D9B39307F00FE300F9F217
:10674000B307AF008583FDB53304E541AE8481BB5B
:10675000E31D0FFCE30505E8AE84BDBD854725BDFF
:10676000854749BF0149E39707EC814E814779B3DB
:10677000B307E5414289AE8419BBB28741B3328E7B
:1067800042897DBD054735BF370680001357750127
:106790009307F6FF1377F70F9305E007B3F6A7000B
:1067A0009357F50163FCE5009305D00963FAE50012
:1067B000370500801345F5FF3E95828001458280B4
:1067C00093055009D18E63CDE500130660093307A8
:1067D000E64033D7E6003305E040F5F33A858280A2
:1067E0001307A7F63397E600FDB713577501370671
:1067F00080009307F6FF1377F70F9305E007B3F6D2
:10680000A7009357F501014563F4E50099C3828021
:1068100082809307E0097D55E3EBE7FE930550097D
:10682000B3E7C60063D7E5001307A7F63395E70083
:106830008280130560093307E54033D5E700828085
:10684000411106C622C426C20DCD9357F54133C46B
:10685000A7001D8CAA842285492E9307E00933875F
:10686000A74093076009FD8063CCE702A1469377B8
:10687000F70F63D5A60061153314A4002604258004
:1068800021A0814481470144260413559400B2405D
:106890002244DE07FE045D8D458D924441018280D5
:1068A0009307900963DDE7009307B5019546B31799
:1068B000F400898E3354D400B337F0005D8C9547D3
:1068C00063D6A7009307B5FF3314F400B70600FCA6
:1068D000FD16937774003376D40085C39377F40064
:1068E0009145638CB70011069317560063D70700D4
:1068F0009307F009758E3387A7401314660025802F
:106900009377F70F51B7411106C622C415CD2A84DB
:10691000E92C9307E0093387A7409307600963C018
:10692000E704A1469377F70F63D5A60061153314EA
:10693000A40026042580260413559400B240224466
:10694000DE075D8D410182800144260413559400C9
:10695000B24022448147DE075D8D4101828093076A
:10696000900963DDE7009307B5019546B317F4007E
:10697000898EB337F0003354D4005D8C954763D6CD
:10698000A7009307B5FF3314F400B70600FCFD160B
:10699000937774003376D40085C39377F4009145E0
:1069A000638CB70011069317560063D7070093074F
:1069B000F009758E3387A7401314660025802604DE
:1069C00013559400B24022449377F70FDE075D8D94
:1069D00041018280135775011377F70F4111930717
:1069E000170022C426C21314950006C693F7E70FBA
:1069F00025809354F50185C7935734001307073852
:106A00007604B2075207B1831395F401D98FC98F69
:106A1000B240228522449244BE854101828005EB2A
:106A200039C42285D922A94763C6A7042D47098FF7
:106A3000930755013357E4003314F4009317C7004C
:106A400013079038098FB1831377F77F5DBF01CCAF
:106A500013573400B7070800D98FB2077604B18303
:106A60001307F07F79BF1307F07F814759BF0147B4
:106A7000814741BF130755FF3317E40001447DBF31
:106A800093D645019397C50093F6F67FB18313869D
:106A900016008E071357D5011376E67FFD815D8FB3
:106AA0009318350035CE138806C89307E00F63DDD1
:106AB00007018147139597009306F00FDE062581A5
:106AC000FE05558D4D8D82806355000B9317650033
:106AD0000E07B337F000D98F93D8D801B3E7170169
:106AE00013F777006301071013F7F700914663036C
:106AF000D7009107370700047D8F75C7130718006B
:106B00001306F00F9376F70FE305C7FA9A07A583EC
:106B100013959700DE062581FE05558D4D8D8280EB
:106B2000B367170199EE85CF95479A07A58313950B
:106B3000970093F6F60FDE062581FE05558D4D8DE7
:106B40008280A5DBB7074000139597009306F00FEE
:106B5000DE0681452581FE05558D4D8D828081475C
:106B6000139597008146DE062581FE05558D4D8DD6
:106B70008280A5576348F804F94737068000B38739
:106B800007417D45598E6351F50479573307074115
:106B9000130500023357E6006388A700938626CAD0
:106BA000B316D600B3E8D800B3371001D98F13F766
:106BB0007700014815FB139757008546E34807F413
:106BC0008146A5B781468DB7938626C83397D800EE
:106BD0003337E000B316D600B3D8F800B367D70058
:106BE000B3E7F800E9B7C28689B7C167637CF502ED
:106BF0009307F00F1307000263EBA700972700002D
:106C000093878715AA9788233305A740828021811F
:106C10009727000093874714AA9788236147330575
:106C2000A7408280B7070001636DF5006181972757
:106C3000000093876712AA97882321473305A7404E
:106C4000828041819727000093870711AA978823A4
:106C500041473305A7408280B3C7A5008D8B33071A
:106C6000C50081E78D4763EDC700AA87637EE5080D
:106C7000942185078505A38FD7FEE3EBE7FE82808D
:106C800093763500AA8789CA942185078505A38F45
:106C9000D7FE93F63700C5BF9376C7FF138606FE6F
:106CA00063F0C70683A3050083A2450083AF850078
:106CB00003AFC50083AE050103AE450103A3850103
:106CC00083A8C5019385450223A0770003A8C5FFCB
:106CD00023A2570023A4F70123A6E70123A8D70185
:106CE00023AAC70123AC670023AE1701938747028D
:106CF00023AE07FF75B790419107910523AEC7FEFC
:106D0000E3EBD7FEE3E6E7F6828039713EDA2ED276
:106D100032D436D63AD842DC46DE9387818122CC03
:106D2000804326CA06CEAA8409C41C4C99E3228556
:106D300005250C4454102686228536C6EF00905B4C
:106D4000F2406244D24421618280011126CA4AC8BD
:106D500006CE22CC4EC652C4AA842E8901C51C4D33
:106D600091E3FD239C4C804499E32685D523972706
:106D7000000093876710631BF402C0405E24A18B60
:106D8000B1C71C48A1C7FD59294A1C4483450900C5
:106D9000FD17B1E91CC463DD07062286A9452685D7
:106DA0007522FD576308F502294535A09727000095
:106DB0009387870E6314F4008044C9B797270000B7
:106DC00093878709E31CF4FAC0444DBFA28526854A
:106DD000252C55D97D55F2406244D2444249B249EE
:106DE000224A056182801CC4050963D70700184C3C
:106DF00063CAE700638845011C401387170018C069
:106E00008CA361B7228626859122E31035F9D9B784
:106E10001C401387170018C0294798A371B79387A0
:106E20008181AA8588436FF05FF241119387818148
:106E300022C4804326C206C61C5CAA8495EB614529
:106E4000EF000077B737CDAB08DC9387E7301CC184
:106E5000B7176DE6938747235CC1B7E705009387B3
:106E6000C7EE1CC5AD475EA50547814718C95CC97B
:106E70001C5CB240224484CB23AA07009244410107
:106E8000828041119387818122C4804306C61C5CA5
:106E90008DEB6145312FB737CDAB08DC9387E730F9
:106EA0001CC1B7176DE6938747235CC1B7E70500A0
:106EB0009387C7EE1CC5AD475EA50547814718C936
:106EC0005CC9105C3787954CB7F75158144A484A4B
:106ED0001307D7F29387D742B387F602B240224412
:106EE0003305E5023E95B387E60233B7E6029386A3
:106EF000170014CA2A9733B5F6003A9548CA060512
:106F000005814101828035713ECBB707008093C770
:106F1000F7FF3ECE3EC8C1779387872032C536C77C
:106F20003AC942CD46CF3ECA938781812AC42ACC32
:106F3000884334012E862C0086DE36C2EF00500EC8
:106F4000A24723800700F6500D618280011122CCF8
:106F500026CA4AC806CE4EC6AA842E89328401C5E6
:106F60001C4D91E3F526972700009387E7F0631700
:106F7000F406C0401C4C1CC45E24A18BC1C31C4839
:106F8000B5CF1C4808409379F90F1379F90F1D8D7F
:106F90005C486346F500A2852685692C25E51C44DE
:106FA0000505FD171CC41C401387170018C023805B
:106FB00037015C486388A7005E24858B81CBA94795
:106FC0006316F900A2852685B5240DEDF2406244D2
:106FD0004A85D2444249B249056182809727000020
:106FE000938787EB6314F400804469B79727000008
:106FF000938787E6E310F4F8C044ADBFA2852685E9
:10700000212041D17D59D9B741119387818126C271
:10701000844322C44AC006C62A892E8489C49C4C53
:1070200099E326853526972700009387E7E4631BBD
:10703000F402C0400317C40093170701C18393F6FD
:107040008700ADEA93F6070195EEA5472320F900E6
:10705000136707045AA47D55B24022449244024962
:107060004101828097270000938707E36314F400AF
:107070008044C9B797270000938707DEE31CF4FA22
:10708000C0444DBF918B9DC34C5889C9930744049C
:107090006384F5004A851523232A04025E242322F3
:1070A000040093F7B7FD5EA41C481CC05E2493E760
:1070B00087005EA41C4899EB5E241307002093F719
:1070C00007286385E700A2854A8591295E2413F786
:1070D00017001DC35C4823240400B307F0401CCCF8
:1070E0001C480145B5FB8317C40013F707082DD7CB
:1070F00093E707045EA485B7898B014791E358485D
:1071000018C4F9BFDE25011122CC26CA06CE4AC812
:107110004EC613F78700AA842E8479EBD841634DBD
:10712000E000B841634AE0000145F2406244D244C5
:107130004249B2490561828058547DD703A90400B1
:107140009396370123A0040063DB060670485E2493
:10715000918B99C75C401D8E5C5899C33C401D8E35
:107160005C540C50814626858297FD575A24631D36
:10717000F5009440F54763E8D706B7074020850738
:10718000B3D7D700858BA5C31C48232204001CC09D
:107190009317370163D80700FD576314F5009C402F
:1071A00091E368C84C5823A02401BDDD9307440433
:1071B0006384F50026851121232A0402B5B70C50FB
:1071C0000146854626850297FD572A86E311F5F884
:1071D0009C40B5DF75476385E70059476393E70433
:1071E00023A0240191B7136707045AA47D5535BF26
:1071F00083A90501E38A09F203A905008D8B23A069
:10720000350133093941014791E3D84918C4E35D99
:1072100020F11C540C50CA864E86268582976347FF
:10722000A0005E2493E707045EA4C9B7AA993309B6
:10723000A940F1BF9C49A5C3011122CC06CE2A84E6
:1072400011C51C4D81E72EC62122B24597270000AB
:10725000938787C2639CF5004C408397C5009DC708
:1072600022856244F24005616FF0DFE99727000054
:10727000938787C26394F5000C44C5B79727000035
:10728000938787BDE39BF5FC4C44C1BFF240624449
:1072900001450561828001458280411122C406C6F4
:1072A0002A844EA572A5232005002322050023244D
:1072B00005002322050623280500232A0500232C88
:1072C0000500214681451305C505EF807FED971721
:1072D00000009387E7E85CD097170000938707EBDF
:1072E0001CD4971700009387E7EE5CD49717000033
:1072F000938747F100D01CD8B240224441018280DC
:1073000097050000938545F391AA411126C2130603
:1073100080069384F5FFB384C4024AC02E8922C438
:1073200006C693854407352E2A8401CD2320050007
:1073300023222501310508C4138684068145EF8088
:107340003FE62285B24022449244024941018280B4
:107350001C4DA5E7411106C622C49707000093877C
:1073600067FA1CD59387C1819C43232405042326F7
:107370000504232805046314F50085471CCD2A84E1
:10738000352848C022851D2808C42285052848C400
:10739000484001469145EFF05FF008440546A54599
:1073A000EFF0BFEF48440946C945EFF01FEF8547AE
:1073B0001CCCB240224441018280828041119387DB
:1073C000C18126C284434AC006C69C4C22C42A8975
:1073D00081E72685EFF0DFF7938484048044DC4066
:1073E000FD1763D607009C40B9CF8440C5BF031783
:1073F000C40039E7C177850723220406232004004F
:1074000023220400232404005CC423280400232A2C
:107410000400232C0400214681451305C405EF8098
:107420003FD8232A0402232C040223240404232605
:1074300004042285B24022449244024941018280E0
:107440001304840671BF91454A85EFF01FEC88C094
:1074500049FDB1472320F9000144E1BF797122D4ED
:107460004AD052CC56CA5AC85EC606D626D24ECE8E
:107470002A8AAE8A130485040149054BFD5B09EC99
:10748000B25022544A8592540259F249624AD24A71
:10749000424BB24B45618280044483294400FD196C
:1074A00063D409000040E1BFDE24637BFB008397C7
:1074B000E40063877701A6855285829A3369A90023
:1074C00093848406E9BF1971A6DAAE848395E5003A
:1074D000A2DC86DE328463DB0500DE2423A0060006
:1074E00093F7070885E7930700401DA0300836C6CC
:1074F000EF00D057B246E34205FE7247BD67F98FF1
:107500007977BA9793B717009CC2F1BF930700042D
:107510001CC0F6506654D654014509618280DE25B0
:10752000011122CC06CE26CA4AC8898B2E8489CF67
:10753000930774041CC01CC885475CC8F2406244B1
:10754000D24442490561828074003000AA84EFF081
:107550009FF7A2452A892685292219E98317C400A5
:1075600013F7072061FFF19B93E727005EA4C9B7DB
:1075700097070000938707D99CD45E2408C008C8E9
:1075800093E707085EA4A2475CC8B24781CF831582
:10759000E4002685EF00B05011C55E24F19B93E70F
:1075A00017005EA45E243369F9002316240179B71D
:1075B00093878181AA8588436DA0DDC183A7C5FF1C
:1075C000411122C406C626C21384C5FF63D3070037
:1075D0003E94AA84EF00D0589387C18A9C4381EFE0
:1075E0002322040023A6818A2244B24026859244A5
:1075F00041016F001057637EF40014403307D4003C
:107600006396E7009843DC43369718C05CC0D9BF47
:10761000BA87D84319C3E37DE4FE94433386D70089
:10762000631F86001040B29694C33386D700E31DD3
:10763000C7FA10435843B29694C3D8C375B763755D
:10764000C400B1479CC04DB71040B306C4006316D8
:10765000D70014435843B29614C058C0C0C369B78A
:107660008280011126CA93843500F19806CE22CC7F
:107670004AC84EC6A104B14763F5F404B14463E4BB
:10768000B4042A89EF00D04D9387C18A98433A8485
:1076900029E49387018B9C4399E781454A85EF0054
:1076A000D02823A8A18AA6854A85EF001028FD5975
:1076B00063193507B1472320F9004A85EF00704A66
:1076C00029A0E3DE04FAB1471CC10145F24062443F
:1076D000D2444249B249056182801C40858F63CF04
:1076E0000702AD4663F6F6001CC03E9404C031A00C
:1076F0005C406313870223A6F18A4A85EF00704637
:107700001305B4009307440061993307F5405DDF2A
:107710003A94898F1CC05DBF5CC3C5B722874040C7
:1077200085BF130435007198E30285FCB305A440BE
:107730004A85EF00901FE31B35FBADBF01114AC81E
:1077400003A9850022CC52C45AC006CE26CA4EC612
:1077500056C22E84328B368A63E92609DE2513F75A
:10776000074851C304408C495848AA8AB389B44099
:107770008D44B384E4020947B3C4E40213871600BE
:107780004E9763F3E400BA8493F70740BDCFA68514
:107790005685EFF01FED2A891DE1B14723A0FA00BD
:1077A0005E247D5593E707045EA4F2406244D24410
:1077B0004249B249224A924A024B056182800C48F2
:1077C0004E86EFF06FC95E2493F7F7B793E707088B
:1077D0005EA42328240144C84E99B3843441232055
:1077E000240104C4528963732A01528908404A86DD
:1077F000DA85EF0090321C440145B38727411CC451
:107800001C403E99232024014DB726865685EF0063
:1078100070352A895DFD0C485685EFF01FDAB5BF3B
:10782000DE25717126D34AD14ECF06D722D552CD4F
:1078300056CB5AC95EC762C566C393F70708AA89C3
:107840002E89B284B9C39C49A9E39305000436C6C6
:10785000EFF03FE12320A9002328A900B24615E15B
:10786000B14723A0F9007D55BA502A549A540A59B9
:10787000FA496A4ADA4A4A4BBA4B2A4C9A4C4D6149
:10788000828093070004232AF90093070002A30CC7
:10789000F1029307000302DA230DF10236CE930BB7
:1078A0005002971A0000938A2A61054C294B2684BE
:1078B0001C2099C363997709B30C9440638E0C0024
:1078C000E6862686CA854E85EFF05FE7FD57630B97
:1078D000F518D256E69636DA1C2063850718FD5750
:1078E0009304140002D002D63ED202D4A3010106B2
:1078F00082DC8C2015465685EF00B02013841400DE
:10790000825721E513F7070109C713070002A301F6
:10791000E10613F7870009C71307B002A301E106C8
:1079200094201307A002638AE602B2572684814698
:107930002546182093051400130707FD6372E60619
:107940008DC63ED61DA00504A5B733055541331598
:10795000AC00C98F3ED0A28469BF7247930647002E
:10796000184336CE634707023AD618209307E00241
:10797000631DF70418309307A002631BF702F24758
:107980000904138747009C433ACE63C107023ED2E5
:107990002DA83307E04093E727003AD63ED0F1B751
:1079A000B387670385462E84BA9761B7FD57C5B77D
:1079B000050402D28146814725461820930514000C
:1079C000130707FD6376E606F9F20C200D4617153E
:1079D00000001305E54EEF00D01211CD97170000FF
:1079E0009387074E1D8D93070004B397A700025598
:1079F00005045D8D2AD00C201946171500001305CB
:107A0000654C93041400230CB102EF00900F25C5C0
:107A10009787FFFF9387075F95E70257F247137732
:107A2000071009CF91073ECED257D2973EDA41B523
:107A3000B387670385462E84BA9741B79D07E19BBC
:107A4000A107D5B7780897060000938666CF4A86C7
:107A50000C104E8597000000E7000000FD572A8AB1
:107A6000E314F5FC8357C9007D5593F70704E39DA4
:107A700007DE5255D5BB780897060000938646CCA2
:107A80004A860C104E850921D1BF1C46FD171CC625
:107A900063DA0700184E63C5E700A9476394F50051
:107AA0006FF0CFCA1C422E851387170018C28CA313
:107AB0008280011122CC26CA4AC84EC652C406CEC4
:107AC0002A89AE893284B304D6007D5A63149400A7
:107AD000014509A80C204E864A85EFF01FFB0504DE
:107AE000E31645FFF2406244D2444249B249224A79
:107AF00005618280357122CD26CB4AC94EC706CF9B
:107B000052C556C35AC1DEDEE2DCE6DAAA89AE848B
:107B10003289368409C51C4D99E3EFF07F839717AE
:107B20000000938767356398F40C83A44900DE2432
:107B3000A18BE5C79C48F5C393070002A304F1029B
:107B40009307000302D22305F10222C6930B5002D1
:107B5000971A0000938A4A36054C294B4A841C2008
:107B600099C3639F770DB30C2441638E0C00E686A6
:107B70004A86A6854E85EFF0DFF3FD57630FF51CAF
:107B80009256E69636D21C206389071CFD571309CE
:107B9000140002C802CE3ECA02CCA309010482D45A
:107BA0008345090015465685A92F13041900C247BD
:107BB00051E913F7070109C713070002A309E104FC
:107BC00013F7870009C71307B002A309E10483462E
:107BD00009001307A002638FE606F2474A84814634
:107BE0002546182093051400130707FD6377E60A5E
:107BF000B5CA3ECE85A8971700009387E7296395FD
:107C0000F40083A4890025B7971700009387C72441
:107C1000E39FF4F083A4C90019BFA6854E85EFF059
:107C2000AFBE19D97D55FA406A44DA444A49BA4987
:107C30002A4A9A4A0A4BF65B665CD65C0D618280E2
:107C4000050431BF330555413315AC00C98F3EC81B
:107C50002289B9B7324793064700184336C66347AF
:107C600007023ACE18209307E002631DF70418308C
:107C70009307A002631BF702B2470904138747006A
:107C80009C433AC663C107023ECA2DA83307E040B1
:107C900093E727003ACE3EC8F1B7B387670385461E
:107CA0002E84BA973DBFFD57C5B7050402CA814669
:107CB00081472546182093051400130707FD6374B8
:107CC000E606F9F20C200D46171500001305451FB6
:107CD0000D2D11CD971700009387871E1D8D9307DB
:107CE0000004B397A700424505045D8D2AC80C2007
:107CF0001946171500001305E51C13091400230489
:107D0000B102012535C19787FFFF9387A72F95E71C
:107D10004247B2471377071009CF91073EC69257E3
:107D2000D2973ED225BDB387670385462E84BA9786
:107D300051B79D07E19BA107D5B7780097060000D2
:107D4000938666D726860C084E8597000000E700CC
:107D50000000FD572A8AE314F5FCDE2493F707049C
:107D6000E39207EC1255C1B57800970600009386A0
:107D700086D426860C084E85012AE1BF797156CA41
:107D80009C49BA8A984522D426D24ECE52CC06D6E9
:107D90004AD05AC85EC6AA892E84B284368A63D372
:107DA000E700BA879CC00347340419C385079CC009
:107DB0001C4093F7070281C79C4089079CC0032998
:107DC000040013796900631A0900130B9401FD5B29
:107DD0005C449840998F634CF9041C4083463404FA
:107DE00093F70702B336D000A5EB13063404D2850F
:107DF0004E85829AFD576303F5041C401146984056
:107E0000998B544481446397C700B384E64063D39D
:107E1000040081441C4418486354F700998FBE94B1
:107E2000014969047D5B63982405014509A88546DD
:107E30005A86D2854E85829A631E75017D55B25051
:107E4000225492540259F249624AD24A424BB24BEE
:107E5000456182800509ADBF3307D40013060003D6
:107E6000A301C7040347540493871600A297890609
:107E7000A381E7049DBF85462286D2854E85829ADE
:107E8000E30E65FB050945B7797122D426D24AD0A5
:107E90004ECE06D652CC56CA5AC8B689942D9307F0
:107EA00090063289AA842E8413863504638DF602E7
:107EB00063E2D706930780056386F61863EDD70063
:107EC000638E062093073004638EF60A930A240417
:107ED0002301D404C9A0930730066385F60A9307EB
:107EE0004006E395F6FE1C40084393F60708930509
:107EF0004500C5C61C410CC363D807001307D00258
:107F0000B307F040A301E40497160000938606FC33
:107F1000294765A8930700076382F61663E5D70231
:107F20009307E0066389F6189307F006E390F6FAE4
:107F30000C401C4313F80508138547006307080627
:107F400008C39C4385A893075007E383F6FE930775
:107F500080076389F61293073007E399F6F61C430E
:107F6000D04181459386470014C383AA07005685F4
:107F7000492E01C53305554148C05C401CC8A301CA
:107F8000040461A81C43930A2404938647009C437D
:107F900014C32301F4048547D5B793F607041C41A5
:107FA0000CC3B9DAC207C18781BF93F5050408C3C2
:107FB000C9D99E231307F0066387E60E97160000C3
:107FC0009386C6F02947A30104044C400CC463C542
:107FD000050008406D9908C099E3B28A89CDB28A3C
:107FE000B3F5E702FD1AB6958C212380BA00B3D50C
:107FF000E70263F0E70CA147631EF7001C40858B86
:1080000091CB58401C4863C7E70093070003A38F38
:10801000FAFEFD1A3306564110C84E87CA86700014
:10802000A2852685EFF09FD57D5A631D450B7D55B2
:10803000B250225492540259F249624AD24A424BF7
:1080400045618280A382D50497160000938606E8D6
:108050000C40084313F805081C411105630D080284
:1080600008C313F7150001C793E505020CC041478B
:10807000B9FB0C4093F5F5FD0CC0B1B79C4193E7FB
:1080800007029CC193078007A302F404971600001F
:10809000938606E575BF13F8050408C3E30308FCDF
:1080A000C207C1837DBF97160000938626E2214751
:1080B00019BFAE8735B794411C43CC4913F8060865
:1080C000138547006306080008C39C438CC339A08E
:1080D00008C393F606049C43F5DA8EA32328040014
:1080E000B28A25BF14485686CA8526858299E30040
:1080F00045F51C40898B8DE7B2474844E35AF5F2B9
:108100003E853DB785465686CA8526858299E30019
:1081100065F3050A5C443247998FE345FAFEE9BFEF
:10812000014A930A94017D5BF5B7411122C42A8468
:108130002E859797FF1F23A9073E06C6EF909FDF66
:10814000FD576319F5009797FF1F9387E73D9C4301
:1081500091C31CC0B240224441018280411122C41B
:108160002E848395E50006C6912C634905007C4862
:10817000AA977CC8B2402244410182805E247D7768
:108180007D17F98F5EA4FDB7DE25011122CC26CA2A
:108190004AC84EC606CE93F70710AA842E843289A9
:1081A000B68991C78395E500894601460D225E2474
:1081B0007D777D17F98F5EA48315E4006244F24059
:1081C000CE864A86B24942492685D244056125A811
:1081D000411122C42E848395E50006C6CD28FD57A3
:1081E0005A24631AF500FD77FD17F98F5EA4B2409B
:1081F0002244410182808567D98F5EA468C8C5BFCB
:108200008395E50025A8411122C42A842E85B285D4
:1082100036869797FF1F23A9073006C6EF90BFCD7C
:10822000FD576319F5009797FF1F9387E72F9C432E
:1082300091C31CC0B240224441018280411122C43A
:108240002A842E859797FF1F23A0072E06C65D2A36
:10825000FD576319F5009797FF1F9387E72C9C4301
:1082600091C31CC0B240224441018280411122C40A
:108270002A842E85B2859797FF1F23A7072A06C653
:10828000512AFD576319F5009797FF1F9387C72958
:108290009C4391C31CC0B2402244410182804111E1
:1082A00022C42A842E859797FF1F23AF072606C670
:1082B000952AFD576319F5009797FF1F9387C726E7
:1082C0009C4391C31CC0B2402244410182804111B1
:1082D00022C42A842E85B28536869797FF1F23A550
:1082E000072406C6812AFD576319F5009797FF1FDB
:1082F000938787239C4391C31CC0B2402244410111
:10830000828093F5F50F2A966314C500014582809B
:108310001C21E38EB7FE0505C5BF63F1A504B38636
:10832000C500637DD5029345F6FF8147FD17639332
:10833000F50082803387F600034807003387C700C3
:108340002A9723000701DDB73387F500142333078D
:10835000F500850714A3E319F6FE82808147E5BF87
:108360008280828081E5B2856FF0AFAF011122CCAF
:1083700006CE26CA4AC84EC6328401EEEFF0EFA3FD
:108380000149F24062444A85D2444249B2490561FA
:108390008280AE84AA89A9282689E37485FEA285F5
:1083A0004E85EFF00FAC2A8969DDA6852286EFE0C5
:1083B000BF8AA6854E85EFF04FA0E1B7411122C4D8
:1083C0002A842E85B28536869797FF1F23AE071421
:1083D00006C68D28FD576319F5009797FF1F9387F1
:1083E000A7149C4391C31CC0B24022444101828027
:1083F00083A7C5FF1385C7FF63D50700AA959C41D6
:108400003E958280930780051797FF1F232EF71054
:108410007D558280930780051797FF1F2326F7104D
:108420007D558280930780051797FF1F232EF70E37
:1084300001458280930780051797FF1F2326F70EBB
:108440007D558280930780051797FF1F232EF70C19
:108450007D55828053797374656D436C6B3A2564E6
:108460000D0A00004368697049443A253038780D98
:108470000A00000043616C696272617474696F6E16
:108480005F56616C203A2025640A0000CDCC4C3D3B
:108490006666663F0000F0439A9999999999A93FB9
:1084A000CDCCCCCCCCCCEC3F696E2074696D312046
:1084B000697271200000000000F07F45000000009C
:1084C0000000000000000440000000000000204008
:1084D000000000000000E03F000000000000344009
:1084E00000000000CF4636400000006066661A407B
:1084F0001D130F130213F412E612D712C812B91289
:10850000AA129A128A127A126A1259124812371251
:10851000251213120112EE11DB11C811B511A111B0
:108520008D11791164114F113A1125110F11F910A4
:10853000E310CC10B5109E1087106F1057103F102D
:1085400026100D10F40FDB0FC20FA80F8E0F740F43
:10855000590F3F0F240F090FED0ED20EB60E9A0ED3
:108560007E0E620E460E290E0C0EF00DD30DB60DCA
:10857000980D7B0D5E0D400D220D050DE70CC90C0D
:10858000AB0C8D0C6F0C510C330C150CF70BD90B7D
:10859000BB0B9C0B7E0B600B420B240B060BE80AFB
:1085A000CA0AAD0A8F0A710A540A360A190AFC0966
:1085B000DF09C209A50988096C094F0933091709A0
:1085C000FB08DF08C308A8088D08720857083C0894
:1085D00021080708ED07D307B907A00786076D072D
:1085E00054073C0723070B07F306DB06C406AD065A
:1085F00096067F06680652063C0626061006FB0510
:10860000E605D105BC05A70593057F056B05580553
:10861000450532051F050C05FA04E804D604C40418
:10862000B304A10490047F046F045F044E043E046D
:108630002F041F0410040104F203E303D503C7034E
:10864000B903AB039D0390038203750368035C03C6
:108650004F03430336032A031F0313030703FC02DC
:10866000F102E602DB02D102C602BC02B202A7029C
:108670009E0294028A02810277026E0265025C0207
:1086800054024B0242023A0232022A0222021A0227
:1086900012020B020302FC01F401ED01E601DF010D
:1086A000D801D201CB01C401BE01B801B101AB01B7
:1086B000A5019F01990194018E01880183017D012B
:1086C000780173016E01690163015E015A01550170
:1086D0005001000000401C460000C84200009041CC
:1086E00000008041000000419A9999999999C93FE9
:1086F0009A9999999999B93F466C6F6174493A2052
:108700002564202F20313030200A00006E6F776FF3
:10871000726B200017B75138ACC5273700007A4478
:108720000AD7A33B000000006666666666662C40BA
:108730005B494E464F5D205B25733A25645D2052B0
:108740006567697374726174696F6E2073756363B2
:10875000657373200D0A0D0A000000005B4552523C
:108760004F525D205B25733A25645D20205265677A
:1087700069737465725F4E756D62657220657272A1
:108780006F723A2578200D0A0D0A00005B4552529F
:108790004F525D205B25733A25645D20205265674A
:1087A00069737465725F53746172745F416464725B
:1087B000657373206572726F72203A202578200DE0
:1087C0000A0D0A00696E2077726974652072656708
:1087D00069737465722000005B494E464F5D205BF3
:1087E00025733A25645D2020534C5F5265616452C5
:1087F0006567697374657242617474657279566FE6
:108800006C74616765200D0A000000005B494E46EC
:108810004F5D205B25733A25645D2020534C5F52E9
:1088200065616452656769737465724368617267F4
:1088300043757272656E74200D0A00005B494E46E6
:108840004F5D205B25733A25645D2020534C5F52B9
:1088500065616452656769737465724469736368BE
:1088600061726743757272656E74200D0A000000B4
:108870005B494E464F5D205B25733A25645D2020A1
:10888000534C5F52656164526567697374657244E5
:10889000697363686172674D6F73537461746520A7
:1088A0000D0A0000000020415B494E464F5D205BF1
:1088B00025733A25645D2020534C5F5265616452F4
:1088C0006567697374657248696768536964654D63
:1088D0006F7354656D7065726174757265200D0AF1
:1088E000000000005B494E464F5D205B25733A2532
:1088F000645D2020534C5F52656164526567697303
:108900007465724D5050544D6F6465200D0A00001F
:108910005B494E464F5D205B25733A25645D202000
:10892000534C5F5265616452656769737465725335
:108930006F6C61724F70656E4369726375697456CE
:108940006F6C74616765200D0A0000005B494E463C
:108950004F5D205B25733A25645D204D617463682B
:108960005F5374617274666C6167207375636365CD
:108970007373200D0A0D0A005B494E464F5D205B64
:1089800025733A25645D204D617463685F6164649A
:10899000726573732073756363657373200D0A0DBD
:1089A0000A0000005B494E464F5D205B25733A2567
:1089B000645D204D617463685F42726F61646361DE
:1089C0007374616464726573732073756363657334
:1089D000730D0A0D0A0000005B494E464F5D205B97
:1089E00025733A25645D20526561645F526567694D
:1089F000737465720D0A0D0A000000005B494E4653
:108A00004F5D205B25733A25645D2057726974655C
:108A10005F52656769737465720D0A0D0A00000084
:108A20005B494E464F5D205B25733A25645D204FC0
:108A300074686572206672616D65730D0A0D0A00B7
:108A40005B494E464F5D205B25733A25645D2042AD
:108A5000726F6164636173745F5363616E0D0A0DBD
:108A60000A0000005B494E464F5D205B25733A25A6
:108A7000645D20526567697374726174696F6E5FBB
:108A8000726571756573740D0A0D0A005B494E4677
:108A90004F5D205B25733A25645D2066756E636FBC
:108AA0006465206572726F722025780D0A0D0A00C8
:108AB00020647574795F726174696F203A2025644F
:108AC0002F31303030200A0020496E7075745F56A7
:108AD0006F6C74616765203A2025642F3130302037
:108AE0000A00000020766F7574203A2025642F312B
:108AF0003030200A000000002076426174746572F4
:108B000079203A2025642F313030200A00000000FF
:108B100020496F7574203A2025642F313030200AA7
:108B20000000000020496469736F7574203A2025A5
:108B3000642F313030200A00206D6F7354203A20AA
:108B400025642F3130200A0020696D706564616EE4
:108B50006365203A2025642F31303030200A000030
:108B600020675F696D706564616E636553746172DF
:108B700074203A202564200A00000000206D6F73E5
:108B80005374617465203A202564200A00000000B7
:108B900020626174746572795374617465203A203F
:108BA0002564200A00000000206F75747075744100
:108BB0006761696E466C6167203A202564200A006F
:108BC000206578636573736976654C6F6164466C84
:108BD0006167203A202564200A00000020302EC35F
:108BE000BBD3D0B9A4D7F73B20312EE4B8C1F7C42A
:108BF000A3CABD3B20322EBAE3C1F7C4A3CABD3B12
:108C000020332EBAE3D1B9C4A3CABD3B20342EB859
:108C1000A1B3E4C4A3CABD3B20352EC3BBD3D0B59A
:108C2000E7B3D8203A202564200A00000000803FE6
:108C3000000040409A99193F9A9999999999B9BF1A
:108C40007B14AE47E17A843F000030410000704160
:108C50003333333F36C3FFFF28C2FFFF28C2FFFF75
:108C600026C2FFFF2EC2FFFF2EC2FFFFF4C1FFFF8F
:108C700026C2FFFF2EC2FFFFF4C1FFFF2EC2FFFF7F
:108C800026C2FFFF22C3FFFF22C3FFFF22C3FFFF55
:108C9000F4C1FFFF72D2FFFF98D1FFFF6CD2FFFF3C
:108CA000A0D1FFFF6CD2FFFF66D1FFFF6CD2FFFFA8
:108CB000A0D1FFFF98D1FFFF98D1FFFF66D1FFFF42
:108CC000A0D1FFFFA6D1FFFFA6D1FFFFA6D1FFFFD6
:108CD00066D1FFFF58D1FFFF58D1FFFF2CD2FFFF15
:108CE00008D3FFFF2CD2FFFF26D1FFFF2CD2FFFFBE
:108CF00008D3FFFF58D1FFFF58D1FFFF26D1FFFF58
:108D000008D3FFFF66D1FFFF66D1FFFF66D1FFFFEB
:108D100026D1FFFFDCD5FFFF2AD5FFFF2AD5FFFFB5
:108D200028D5FFFF2ED5FFFF2ED5FFFFFED4FFFF76
:108D300028D5FFFF2ED5FFFFFED4FFFF2ED5FFFF66
:108D400028D5FFFFCAD5FFFFCAD5FFFFCAD5FFFF51
:108D5000FED4FFFF00010202030303030404040422
:108D600004040404050505050505050505050505B7
:108D70000505050506060606060606060606060697
:108D80000606060606060606060606060606060683
:108D90000606060607070707070707070707070767
:108DA0000707070707070707070707070707070753
:108DB0000707070707070707070707070707070743
:108DC0000707070707070707070707070707070733
:108DD0000707070708080808080808080808080817
:108DE0000808080808080808080808080808080803
:108DF00008080808080808080808080808080808F3
:108E000008080808080808080808080808080808E2
:108E100008080808080808080808080808080808D2
:108E200008080808080808080808080808080808C2
:108E300008080808080808080808080808080808B2
:108E400008080808080808080808080808080808A2
:108E500008080808000000000000000000000000F2
:108E60000000000000000000000000000000000002
:108E700000000000000000000000000000000000F2
:108E800000000000000000000000000000000000E2
:108E900000000000000000000000000000000000D2
:108EA00000000000000000000000000000000000C2
:108EB00000000000232D302B20000000686C4C00C7
:108EC0006566674546470000303132333435363702
:108ED00038394142434445460000000030313233C6
:108EE00034353637383961626364656600000000E6
:108EF000000000000000000001020304060708094A
:108F0000000000000102030401020304060708092F
:108F100000000000000000000000000000E8038CDA
:108F2000051400A406DC05A00564008C050A0001F8
:108F300000140014004600320028000A003C001013
:108F40000E000000534C11111111111111010001FB
:108F50000016000030000000D02D000010000000BE
:108F60005A2B0000A0000000222B0000A1000000EE
:108F7000C22A0000D0000000322D0000D100000005
:108F8000942C000001010000822A00000201000070
:108F9000422A000003010000022A00000401000030
:108FA000C0290000050100007E2900000601000024
:108FB00056290000070100002829000000000000D9
:108FC00003000000802500000000000000000000F9
:108FD000000000000000000000000000040000008D
:108FE00080250000000000000000000000000000DC
:108FF0000000000000000000748E0000948E00004D
:10900000548E00000000000000000000000000007E
:109010000000000000000000000000000000000050
:109020000000000000000000000000000000000040
:109030000000000000000000000000000000000030
:109040000000000000000000000000000000000020
:109050000000000000000000006CDC0202040608B2
:10906000281500200000403F01010101010100001E
:089070000401002004010020AE
:00000001FF
